 j2pkcs11

 Timestamp is 28f31e08 (reproducible build file hash)

 Preferred load address is 0000000180000000

 Start         Length     Name                   Class
 0001:00000000 0000c060H .text$mn                CODE
 0001:0000c060 00000036H .text$mn$00             CODE
 0001:0000c096 00000092H .text$x                 CODE
 0002:00000000 000001a0H .idata$5                DATA
 0002:000001a0 00000038H .00cfg                  DATA
 0002:000001d8 00000008H .CRT$XCA                DATA
 0002:000001e0 00000008H .CRT$XCZ                DATA
 0002:000001e8 00000008H .CRT$XIA                DATA
 0002:000001f0 00000008H .CRT$XIZ                DATA
 0002:000001f8 00000008H .CRT$XPA                DATA
 0002:00000200 00000008H .CRT$XPZ                DATA
 0002:00000208 00000008H .CRT$XTA                DATA
 0002:00000210 00000010H .CRT$XTZ                DATA
 0002:00000218 00000000H .gehcont$y              DATA
 0002:00000218 00000000H .gfids$y                DATA
 0002:00000220 000016e0H .rdata                  DATA
 0002:00001900 00000000H .rdata$CastGuardVftablesA DATA
 0002:00001900 00000000H .rdata$CastGuardVftablesC DATA
 0002:00001900 00000064H .rdata$voltmd           DATA
 0002:00001964 000002bcH .rdata$zzzdbg           DATA
 0002:00001c20 00000008H .rtc$IAA                DATA
 0002:00001c28 00000008H .rtc$IZZ                DATA
 0002:00001c30 00000008H .rtc$TAA                DATA
 0002:00001c38 00000008H .rtc$TZZ                DATA
 0002:00001c40 00000730H .xdata                  DATA
 0002:00002370 000011d8H .edata                  DATA
 0002:00003548 00000078H .idata$2                DATA
 0002:000035c0 00000018H .idata$3                DATA
 0002:000035d8 000001a0H .idata$4                DATA
 0002:00003778 0000040cH .idata$6                DATA
 0003:00000000 00000400H .data                   DATA
 0003:00000400 00000650H .bss                    DATA
 0004:00000000 000008f4H .pdata                  DATA
 0005:00000000 00000060H .rsrc$01                DATA
 0005:00000060 000003a0H .rsrc$02                DATA

  Address         Publics by Value              Rva+Base               Lib:Object

 0000:00000000       __AbsoluteZero             0000000000000000     <absolute>
 0000:00000000       ___safe_se_handler_count   0000000000000000     <absolute>
 0000:00000000       ___safe_se_handler_table   0000000000000000     <absolute>
 0000:00000000       __arm64x_extra_rfe_table   0000000000000000     <absolute>
 0000:00000000       __arm64x_extra_rfe_table_size 0000000000000000     <absolute>
 0000:00000000       __arm64x_native_entrypoint 0000000000000000     <absolute>
 0000:00000000       __arm64x_redirection_metadata 0000000000000000     <absolute>
 0000:00000000       __arm64x_redirection_metadata_count 0000000000000000     <absolute>
 0000:00000000       __dynamic_value_reloc_table 0000000000000000     <absolute>
 0000:00000000       __enclave_config           0000000000000000     <absolute>
 0000:00000000       __guard_check_icall_a64n_fptr 0000000000000000     <absolute>
 0000:00000000       __guard_eh_cont_count      0000000000000000     <absolute>
 0000:00000000       __guard_eh_cont_table      0000000000000000     <absolute>
 0000:00000000       __guard_fids_count         0000000000000000     <absolute>
 0000:00000000       __guard_fids_table         0000000000000000     <absolute>
 0000:00000000       __guard_iat_count          0000000000000000     <absolute>
 0000:00000000       __guard_iat_table          0000000000000000     <absolute>
 0000:00000000       __guard_longjmp_count      0000000000000000     <absolute>
 0000:00000000       __guard_longjmp_table      0000000000000000     <absolute>
 0000:00000000       __hybrid_auxiliary_iat     0000000000000000     <absolute>
 0000:00000000       __hybrid_auxiliary_iat_copy 0000000000000000     <absolute>
 0000:00000000       __hybrid_code_map          0000000000000000     <absolute>
 0000:00000000       __hybrid_code_map_count    0000000000000000     <absolute>
 0000:00000000       __x64_code_ranges_to_entry_points 0000000000000000     <absolute>
 0000:00000000       __x64_code_ranges_to_entry_points_count 0000000000000000     <absolute>
 0000:00000100       __guard_flags              0000000000000100     <absolute>
 0000:00000000       __ImageBase                0000000180000000     <linker-defined>
 0001:00000000       Java_sun_security_pkcs11_Secmod_nssGetModuleList 0000000180001000 f   j2secmod.obj
 0001:0000023c       Java_sun_security_pkcs11_Secmod_nssInitialize 000000018000123c f   j2secmod.obj
 0001:000003d4       Java_sun_security_pkcs11_Secmod_nssVersionCheck 00000001800013d4 f   j2secmod.obj
 0001:00000458       Java_sun_security_pkcs11_Secmod_nssGetLibraryHandle 0000000180001458 f   j2secmod_md.obj
 0001:000004bc       Java_sun_security_pkcs11_Secmod_nssLoadLibrary 00000001800014bc f   j2secmod_md.obj
 0001:0000056c       __local_stdio_printf_options 000000018000156c f i j2secmod_md.obj
 0001:00000574       p11FindFunction            0000000180001574 f   j2secmod_md.obj
 0001:000005f8       snprintf                   00000001800015f8 f i j2secmod_md.obj
 0001:00000650       ckAttributePtrToJAttribute 0000000180001650 f   p11_convert.obj
 0001:00000738       ckAttributeValueToJObject  0000000180001738 f   p11_convert.obj
 0001:0000094c       ckDatePtrToJDateObject     000000018000194c f   p11_convert.obj
 0001:00000a8c       ckSessionInfoPtrToJSessionInfo 0000000180001a8c f   p11_convert.obj
 0001:00000b38       ckVersionPtrToJVersion     0000000180001b38 f   p11_convert.obj
 0001:00000bd4       copyBackPBEInitializationVector 0000000180001bd4 f   p11_convert.obj
 0001:00000d74       jAesCtrParamsToCKAesCtrParamPtr 0000000180001d74 f   p11_convert.obj
 0001:00000ef4       jAttributeToCKAttribute    0000000180001ef4 f   p11_convert.obj
 0001:00000fe0       jCCMParamsToCKCCMParamPtr  0000000180001fe0 f   p11_convert.obj
 0001:000011f0       jDateObjectToCKDatePtr     00000001800021f0 f   p11_convert.obj
 0001:000014fc       jEcdh1DeriveParamToCKEcdh1DeriveParamPtr 00000001800024fc f   p11_convert.obj
 0001:000016a8       jEcdh2DeriveParamToCKEcdh2DeriveParamPtr 00000001800026a8 f   p11_convert.obj
 0001:00001938       jGCMParamsToCKGCMParamPtr  0000000180002938 f   p11_convert.obj
 0001:00001b10       jHkdfParamsToCKHkdfParamsPtr 0000000180002b10 f   p11_convert.obj
 0001:00001dc4       jKeyDerivationStringDataToCKKeyDerivationStringDataPtr 0000000180002dc4 f   p11_convert.obj
 0001:00001eb0       jMechParamToCKMechParamPtr 0000000180002eb0 f   p11_convert.obj
 0001:00001f54       jMechParamToCKMechParamPtrSlow 0000000180002f54 f   p11_convert.obj
 0001:0000228c       jMechanismToCKMechanismPtr 000000018000328c f   p11_convert.obj
 0001:00002334       jPbeParamToCKPbeParamPtr   0000000180003334 f   p11_convert.obj
 0001:0000255c       jPkcs5Pbkd2ParamToCKPkcs5Pbkd2ParamPtr 000000018000355c f   p11_convert.obj
 0001:000028ec       jRsaPkcsOaepParamToCKRsaPkcsOaepParamPtr 00000001800038ec f   p11_convert.obj
 0001:00002aa4       jRsaPkcsPssParamToCKRsaPkcsPssParamPtr 0000000180003aa4 f   p11_convert.obj
 0001:00002be4       jSalsaChaChaPolyParamsToCKSalsaChaChaPolyParamPtr 0000000180003be4 f   p11_convert.obj
 0001:00002d6c       jSsl3KeyMatParamToCKSsl3KeyMatParamPtr 0000000180003d6c f   p11_convert.obj
 0001:00002e44       jSsl3MasterKeyDeriveParamToCKSsl3MasterKeyDeriveParamPtr 0000000180003e44 f   p11_convert.obj
 0001:00002ef8       jTls12KeyMatParamToCKTls12KeyMatParamPtr 0000000180003ef8 f   p11_convert.obj
 0001:0000301c       jTls12MasterKeyDeriveParamToCKTls12MasterKeyDeriveParamPtr 000000018000401c f   p11_convert.obj
 0001:00003114       jTlsExtendedMasterKeyDeriveParamToCKTlsExtendedMasterKeyDeriveParamPtr 0000000180004114 f   p11_convert.obj
 0001:0000324c       jTlsMacParamsToCKTlsMacParamPtr 000000018000424c f   p11_convert.obj
 0001:0000338c       jTlsPrfParamsToCKTlsPrfParamPtr 000000018000438c f   p11_convert.obj
 0001:00003584       jVersionToCKVersionPtr     0000000180004584 f   p11_convert.obj
 0001:0000366c       jX942Dh1DeriveParamToCKX942Dh1DeriveParamPtr 000000018000466c f   p11_convert.obj
 0001:00003818       jX942Dh2DeriveParamToCKX942Dh2DeriveParamPtr 0000000180004818 f   p11_convert.obj
 0001:00003ab8       keyMatParamToCKKeyMatParam 0000000180004ab8 f   p11_convert.obj
 0001:00003eec       masterKeyDeriveParamToCKMasterKeyDeriveParam 0000000180004eec f   p11_convert.obj
 0001:000040dc       Java_sun_security_pkcs11_wrapper_PKCS11_C_1Decrypt 00000001800050dc f   p11_crypt.obj
 0001:0000426c       Java_sun_security_pkcs11_wrapper_PKCS11_C_1DecryptFinal 000000018000526c f   p11_crypt.obj
 0001:0000432c       Java_sun_security_pkcs11_wrapper_PKCS11_C_1DecryptInit 000000018000532c f   p11_crypt.obj
 0001:000043b0       Java_sun_security_pkcs11_wrapper_PKCS11_C_1DecryptUpdate 00000001800053b0 f   p11_crypt.obj
 0001:00004540       Java_sun_security_pkcs11_wrapper_PKCS11_C_1Encrypt 0000000180005540 f   p11_crypt.obj
 0001:000046d0       Java_sun_security_pkcs11_wrapper_PKCS11_C_1EncryptFinal 00000001800056d0 f   p11_crypt.obj
 0001:00004790       Java_sun_security_pkcs11_wrapper_PKCS11_C_1EncryptInit 0000000180005790 f   p11_crypt.obj
 0001:00004814       Java_sun_security_pkcs11_wrapper_PKCS11_C_1EncryptUpdate 0000000180005814 f   p11_crypt.obj
 0001:000049a4       Java_sun_security_pkcs11_wrapper_PKCS11_C_1GCMDecryptInitWithRetry 00000001800059a4 f   p11_crypt.obj
 0001:00004a84       Java_sun_security_pkcs11_wrapper_PKCS11_C_1GCMEncryptInitWithRetry 0000000180005a84 f   p11_crypt.obj
 0001:00004b64       Java_sun_security_pkcs11_wrapper_PKCS11_C_1DigestFinal 0000000180005b64 f   p11_digest.obj
 0001:00004c14       Java_sun_security_pkcs11_wrapper_PKCS11_C_1DigestInit 0000000180005c14 f   p11_digest.obj
 0001:00004c90       Java_sun_security_pkcs11_wrapper_PKCS11_C_1DigestKey 0000000180005c90 f   p11_digest.obj
 0001:00004cd8       Java_sun_security_pkcs11_wrapper_PKCS11_C_1DigestSingle 0000000180005cd8 f   p11_digest.obj
 0001:00004e90       Java_sun_security_pkcs11_wrapper_PKCS11_C_1DigestUpdate 0000000180005e90 f   p11_digest.obj
 0001:00004ff4       Java_sun_security_pkcs11_wrapper_PKCS11_C_1GenerateRandom 0000000180005ff4 f   p11_digest.obj
 0001:0000509c       Java_sun_security_pkcs11_wrapper_PKCS11_C_1SeedRandom 000000018000609c f   p11_digest.obj
 0001:00005130       JNI_OnLoad                 0000000180006130 f   p11_general.obj
 0001:00005140       Java_sun_security_pkcs11_wrapper_PKCS11_C_1Finalize 0000000180006140 f   p11_general.obj
 0001:00005178       Java_sun_security_pkcs11_wrapper_PKCS11_C_1GetInfo 0000000180006178 f   p11_general.obj
 0001:00005210       Java_sun_security_pkcs11_wrapper_PKCS11_C_1GetMechanismInfo 0000000180006210 f   p11_general.obj
 0001:00005284       Java_sun_security_pkcs11_wrapper_PKCS11_C_1GetMechanismList 0000000180006284 f   p11_general.obj
 0001:0000533c       Java_sun_security_pkcs11_wrapper_PKCS11_C_1GetSlotInfo 000000018000633c f   p11_general.obj
 0001:000053b4       Java_sun_security_pkcs11_wrapper_PKCS11_C_1GetSlotList 00000001800063b4 f   p11_general.obj
 0001:00005474       Java_sun_security_pkcs11_wrapper_PKCS11_C_1GetTokenInfo 0000000180006474 f   p11_general.obj
 0001:000054ec       Java_sun_security_pkcs11_wrapper_PKCS11_C_1Initialize 00000001800064ec f   p11_general.obj
 0001:00005558       Java_sun_security_pkcs11_wrapper_PKCS11_finalizeLibrary 0000000180006558 f   p11_general.obj
 0001:00005558       _guard_check_icall_nop     0000000180006558 f   MSVCRT:guard_support.obj
 0001:0000555c       Java_sun_security_pkcs11_wrapper_PKCS11_initializeLibrary 000000018000655c f   p11_general.obj
 0001:000055ac       ckInfoPtrToJInfo           00000001800065ac f   p11_general.obj
 0001:00005728       ckMechanismInfoPtrToJMechanismInfo 0000000180006728 f   p11_general.obj
 0001:000057cc       ckSlotInfoPtrToJSlotInfo   00000001800067cc f   p11_general.obj
 0001:00005948       ckTokenInfoPtrToJTokenInfo 0000000180006948 f   p11_general.obj
 0001:00005cdc       fetchClass                 0000000180006cdc f   p11_general.obj
 0001:00005d0c       prefetchFields             0000000180006d0c f   p11_general.obj
 0001:00005dec       Java_sun_security_pkcs11_wrapper_PKCS11_C_1DeriveKey 0000000180006dec f   p11_keymgmt.obj
 0001:00005fe8       Java_sun_security_pkcs11_wrapper_PKCS11_C_1GenerateKey 0000000180006fe8 f   p11_keymgmt.obj
 0001:00006110       Java_sun_security_pkcs11_wrapper_PKCS11_C_1GenerateKeyPair 0000000180007110 f   p11_keymgmt.obj
 0001:000062ac       Java_sun_security_pkcs11_wrapper_PKCS11_C_1UnwrapKey 00000001800072ac f   p11_keymgmt.obj
 0001:000063e4       Java_sun_security_pkcs11_wrapper_PKCS11_C_1WrapKey 00000001800073e4 f   p11_keymgmt.obj
 0001:00006540       Java_sun_security_pkcs11_wrapper_PKCS11_createNativeKey 0000000180007540 f   p11_keymgmt.obj
 0001:000066d4       Java_sun_security_pkcs11_wrapper_PKCS11_getNativeKeyInfo 00000001800076d4 f   p11_keymgmt.obj
 0001:00007128       copyBackTLSPrfParams       0000000180008128 f   p11_keymgmt.obj
 0001:000072b8       ssl3CopyBackKeyMatParams   00000001800082b8 f   p11_keymgmt.obj
 0001:000072e8       tls12CopyBackKeyMatParams  00000001800082e8 f   p11_keymgmt.obj
 0001:00007318       Java_sun_security_pkcs11_wrapper_PKCS11_connect 0000000180008318 f   p11_md.obj
 0001:00007628       Java_sun_security_pkcs11_wrapper_PKCS11_disconnect 0000000180008628 f   p11_md.obj
 0001:00007654       callJCreateMutex           0000000180008654 f   p11_mutex.obj
 0001:0000781c       callJDestroyMutex          000000018000881c f   p11_mutex.obj
 0001:000079e4       callJLockMutex             00000001800089e4 f   p11_mutex.obj
 0001:00007b9c       callJUnlockMutex           0000000180008b9c f   p11_mutex.obj
 0001:00007d54       makeCKInitArgsAdapter      0000000180008d54 f   p11_mutex.obj
 0001:00007ff8       Java_sun_security_pkcs11_wrapper_PKCS11_C_1CopyObject 0000000180008ff8 f   p11_objmgmt.obj
 0001:000080bc       Java_sun_security_pkcs11_wrapper_PKCS11_C_1CreateObject 00000001800090bc f   p11_objmgmt.obj
 0001:00008174       Java_sun_security_pkcs11_wrapper_PKCS11_C_1DestroyObject 0000000180009174 f   p11_objmgmt.obj
 0001:000081bc       Java_sun_security_pkcs11_wrapper_PKCS11_C_1FindObjects 00000001800091bc f   p11_objmgmt.obj
 0001:0000826c       Java_sun_security_pkcs11_wrapper_PKCS11_C_1FindObjectsFinal 000000018000926c f   p11_objmgmt.obj
 0001:000082a4       Java_sun_security_pkcs11_wrapper_PKCS11_C_1FindObjectsInit 00000001800092a4 f   p11_objmgmt.obj
 0001:0000833c       Java_sun_security_pkcs11_wrapper_PKCS11_C_1GetAttributeValue 000000018000933c f   p11_objmgmt.obj
 0001:000085a0       Java_sun_security_pkcs11_wrapper_PKCS11_C_1SetAttributeValue 00000001800095a0 f   p11_objmgmt.obj
 0001:0000863c       Java_sun_security_pkcs11_wrapper_PKCS11_C_1CloseSession 000000018000963c f   p11_sessmgmt.obj
 0001:000086b8       Java_sun_security_pkcs11_wrapper_PKCS11_C_1GetOperationState 00000001800096b8 f   p11_sessmgmt.obj
 0001:00008770       Java_sun_security_pkcs11_wrapper_PKCS11_C_1GetSessionInfo 0000000180009770 f   p11_sessmgmt.obj
 0001:000087dc       Java_sun_security_pkcs11_wrapper_PKCS11_C_1Login 00000001800097dc f   p11_sessmgmt.obj
 0001:00008874       Java_sun_security_pkcs11_wrapper_PKCS11_C_1Logout 0000000180009874 f   p11_sessmgmt.obj
 0001:000088ac       Java_sun_security_pkcs11_wrapper_PKCS11_C_1OpenSession 00000001800098ac f   p11_sessmgmt.obj
 0001:000089ec       Java_sun_security_pkcs11_wrapper_PKCS11_C_1SessionCancel 00000001800099ec f   p11_sessmgmt.obj
 0001:00008a34       Java_sun_security_pkcs11_wrapper_PKCS11_C_1SetOperationState 0000000180009a34 f   p11_sessmgmt.obj
 0001:00008ad4       notifyCallback             0000000180009ad4 f   p11_sessmgmt.obj
 0001:00008c40       putNotifyEntry             0000000180009c40 f   p11_sessmgmt.obj
 0001:00008cf4       removeNotifyEntry          0000000180009cf4 f   p11_sessmgmt.obj
 0001:00008d8c       Java_sun_security_pkcs11_wrapper_PKCS11_C_1Sign 0000000180009d8c f   p11_sign.obj
 0001:00008ee4       Java_sun_security_pkcs11_wrapper_PKCS11_C_1SignFinal 0000000180009ee4 f   p11_sign.obj
 0001:00008fec       Java_sun_security_pkcs11_wrapper_PKCS11_C_1SignInit 0000000180009fec f   p11_sign.obj
 0001:00009070       Java_sun_security_pkcs11_wrapper_PKCS11_C_1SignRecover 000000018000a070 f   p11_sign.obj
 0001:00009230       Java_sun_security_pkcs11_wrapper_PKCS11_C_1SignRecoverInit 000000018000a230 f   p11_sign.obj
 0001:000092b4       Java_sun_security_pkcs11_wrapper_PKCS11_C_1SignUpdate 000000018000a2b4 f   p11_sign.obj
 0001:00009418       Java_sun_security_pkcs11_wrapper_PKCS11_C_1Verify 000000018000a418 f   p11_sign.obj
 0001:000094f4       Java_sun_security_pkcs11_wrapper_PKCS11_C_1VerifyFinal 000000018000a4f4 f   p11_sign.obj
 0001:00009588       Java_sun_security_pkcs11_wrapper_PKCS11_C_1VerifyInit 000000018000a588 f   p11_sign.obj
 0001:0000960c       Java_sun_security_pkcs11_wrapper_PKCS11_C_1VerifyRecover 000000018000a60c f   p11_sign.obj
 0001:000097cc       Java_sun_security_pkcs11_wrapper_PKCS11_C_1VerifyRecoverInit 000000018000a7cc f   p11_sign.obj
 0001:00009850       Java_sun_security_pkcs11_wrapper_PKCS11_C_1VerifyUpdate 000000018000a850 f   p11_sign.obj
 0001:000099b4       ckAssertReturnValueOK      000000018000a9b4 f   p11_util.obj
 0001:000099bc       ckAssertReturnValueOK2     000000018000a9bc f   p11_util.obj
 0001:00009a94       ckBBoolPtrToJBooleanObject 000000018000aa94 f   p11_util.obj
 0001:00009b20       ckByteArrayToJByteArray    000000018000ab20 f   p11_util.obj
 0001:00009b84       ckCharArrayToJCharArray    000000018000ab84 f   p11_util.obj
 0001:00009b84       ckUTF8CharArrayToJCharArray 000000018000ab84 f   p11_util.obj
 0001:00009c4c       ckULongArrayToJLongArray   000000018000ac4c f   p11_util.obj
 0001:00009d14       ckULongPtrToJLongObject    000000018000ad14 f   p11_util.obj
 0001:00009d8c       createLockObject           000000018000ad8c f   p11_util.obj
 0001:00009e08       fprintf                    000000018000ae08 f i p11_util.obj
 0001:00009e4c       freeCKAttributeArray       000000018000ae4c f   p11_util.obj
 0001:00009ea0       freeCKMechanismPtr         000000018000aea0 f   p11_util.obj
 0001:0000a124       getFunctionList            000000018000b124 f   p11_util.obj
 0001:0000a16c       getFunctionList30          000000018000b16c f   p11_util.obj
 0001:0000a1b4       jAttributeArrayToCKAttributeArray 000000018000b1b4 f   p11_util.obj
 0001:0000a304       jBooleanArrayToCKBBoolArray 000000018000b304 f   p11_util.obj
 0001:0000a3fc       jBooleanObjectToCKBBoolPtr 000000018000b3fc f   p11_util.obj
 0001:0000a498       jByteArrayToCKByteArray    000000018000b498 f   p11_util.obj
 0001:0000a558       jByteObjectToCKBytePtr     000000018000b558 f   p11_util.obj
 0001:0000a5e8       jCharArrayToCKCharArray    000000018000b5e8 f   p11_util.obj
 0001:0000a6dc       jCharArrayToCKUTF8CharArray 000000018000b6dc f   p11_util.obj
 0001:0000a7ec       jCharObjectToCKCharPtr     000000018000b7ec f   p11_util.obj
 0001:0000a87c       jIntegerObjectToCKULongPtr 000000018000b87c f   p11_util.obj
 0001:0000a90c       jLongArrayToCKULongArray   000000018000b90c f   p11_util.obj
 0001:0000aa00       jLongObjectToCKULongPtr    000000018000ba00 f   p11_util.obj
 0001:0000aa90       jObjectToPrimitiveCKObjectPtr 000000018000ba90 f   p11_util.obj
 0001:0000af48       jStringToCKUTF8CharArray   000000018000bf48 f   p11_util.obj
 0001:0000b004       p11ThrowIOException        000000018000c004 f   p11_util.obj
 0001:0000b014       p11ThrowNullPointerException 000000018000c014 f   p11_util.obj
 0001:0000b024       p11ThrowOutOfMemoryError   000000018000c024 f   p11_util.obj
 0001:0000b034       p11ThrowPKCS11RuntimeException 000000018000c034 f   p11_util.obj
 0001:0000b044       printDebug                 000000018000c044 f   p11_util.obj
 0001:0000b0d4       putModuleEntry             000000018000c0d4 f   p11_util.obj
 0001:0000b134       updateGCMParams            000000018000c134 f   p11_util.obj
 0001:0000b228       __GSHandlerCheck           000000018000c228 f   MSVCRT:gshandler.obj
 0001:0000b248       __GSHandlerCheckCommon     000000018000c248 f   MSVCRT:gshandler.obj
 0001:0000b2c0       __security_check_cookie    000000018000c2c0 f   MSVCRT:amdsecgs.obj
 0001:0000b2f0       __chkstk                   000000018000c2f0 f   MSVCRT:chkstk.obj
 0001:0000b2f0       _alloca_probe              000000018000c2f0 f   MSVCRT:chkstk.obj
 0001:0000b660       _DllMainCRTStartup         000000018000c660 f   MSVCRT:dll_dllmain.obj
 0001:0000b6a0       __raise_securityfailure    000000018000c6a0 f   MSVCRT:gs_report.obj
 0001:0000b6d4       __report_gsfailure         000000018000c6d4 f   MSVCRT:gs_report.obj
 0001:0000b81c       __security_init_cookie     000000018000c81c f   MSVCRT:gs_support.obj
 0001:0000b8c8       DllMain                    000000018000c8c8 f   MSVCRT:dll_dllmain_stub.obj
 0001:0000b8ec       ?__scrt_initialize_type_info@@YAXXZ 000000018000c8ec f   MSVCRT:tncleanup.obj
 0001:0000b8fc       ?__scrt_uninitialize_type_info@@YAXXZ 000000018000c8fc f   MSVCRT:tncleanup.obj
 0001:0000b908       __local_stdio_scanf_options 000000018000c908 f i MSVCRT:default_local_stdio_options.obj
 0001:0000b910       __scrt_initialize_default_local_stdio_options 000000018000c910 f   MSVCRT:default_local_stdio_options.obj
 0001:0000b92c       __scrt_acquire_startup_lock 000000018000c92c f   MSVCRT:utility.obj
 0001:0000b968       __scrt_dllmain_after_initialize_c 000000018000c968 f   MSVCRT:utility.obj
 0001:0000b99c       __scrt_dllmain_before_initialize_c 000000018000c99c f   MSVCRT:utility.obj
 0001:0000b9b4       __scrt_dllmain_crt_thread_attach 000000018000c9b4 f   MSVCRT:utility.obj
 0001:0000b9dc       __scrt_dllmain_crt_thread_detach 000000018000c9dc f   MSVCRT:utility.obj
 0001:0000b9f4       __scrt_dllmain_exception_filter 000000018000c9f4 f   MSVCRT:utility.obj
 0001:0000ba54       __scrt_dllmain_uninitialize_c 000000018000ca54 f   MSVCRT:utility.obj
 0001:0000ba84       __scrt_dllmain_uninitialize_critical 000000018000ca84 f   MSVCRT:utility.obj
 0001:0000ba98       __scrt_initialize_crt      000000018000ca98 f   MSVCRT:utility.obj
 0001:0000bae4       __scrt_initialize_onexit_tables 000000018000cae4 f   MSVCRT:utility.obj
 0001:0000bb70       __scrt_is_nonwritable_in_current_image 000000018000cb70 f   MSVCRT:utility.obj
 0001:0000bc08       __scrt_release_startup_lock 000000018000cc08 f   MSVCRT:utility.obj
 0001:0000bc2c       __scrt_uninitialize_crt    000000018000cc2c f   MSVCRT:utility.obj
 0001:0000bc58       __scrt_get_dyn_tls_init_callback 000000018000cc58 f   MSVCRT:dyn_tls_init.obj
 0001:0000bc60       __crt_debugger_hook        000000018000cc60 f   MSVCRT:utility_desktop.obj
 0001:0000bc68       __scrt_fastfail            000000018000cc68 f   MSVCRT:utility_desktop.obj
 0001:0000bdb4       _RTC_Initialize            000000018000cdb4 f   MSVCRT:initsect.obj
 0001:0000bdf0       _RTC_Terminate             000000018000cdf0 f   MSVCRT:initsect.obj
 0001:0000be2c       __isa_available_init       000000018000ce2c f   MSVCRT:cpu_disp.obj
 0001:0000bfd8       _get_startup_argv_mode     000000018000cfd8 f   MSVCRT:argv_mode.obj
 0001:0000bfe0       __scrt_is_ucrt_dll_in_use  000000018000cfe0 f   MSVCRT:ucrt_detection.obj
 0001:0000bff0       memcpy                     000000018000cff0 f   vcruntime:VCRUNTIME140.dll
 0001:0000bff6       memset                     000000018000cff6 f   vcruntime:VCRUNTIME140.dll
 0001:0000bffc       __C_specific_handler       000000018000cffc f   vcruntime:VCRUNTIME140.dll
 0001:0000c002       __std_type_info_destroy_list 000000018000d002 f   vcruntime:VCRUNTIME140.dll
 0001:0000c008       strcmp                     000000018000d008 f   ucrt:api-ms-win-crt-string-l1-1-0.dll
 0001:0000c00e       strcat                     000000018000d00e f   ucrt:api-ms-win-crt-string-l1-1-0.dll
 0001:0000c014       strcpy                     000000018000d014 f   ucrt:api-ms-win-crt-string-l1-1-0.dll
 0001:0000c01a       strlen                     000000018000d01a f   ucrt:api-ms-win-crt-string-l1-1-0.dll
 0001:0000c020       _initterm                  000000018000d020 f   ucrt:api-ms-win-crt-runtime-l1-1-0.dll
 0001:0000c026       _initterm_e                000000018000d026 f   ucrt:api-ms-win-crt-runtime-l1-1-0.dll
 0001:0000c02c       _seh_filter_dll            000000018000d02c f   ucrt:api-ms-win-crt-runtime-l1-1-0.dll
 0001:0000c032       _configure_narrow_argv     000000018000d032 f   ucrt:api-ms-win-crt-runtime-l1-1-0.dll
 0001:0000c038       _initialize_narrow_environment 000000018000d038 f   ucrt:api-ms-win-crt-runtime-l1-1-0.dll
 0001:0000c03e       _initialize_onexit_table   000000018000d03e f   ucrt:api-ms-win-crt-runtime-l1-1-0.dll
 0001:0000c044       _execute_onexit_table      000000018000d044 f   ucrt:api-ms-win-crt-runtime-l1-1-0.dll
 0001:0000c04a       _cexit                     000000018000d04a f   ucrt:api-ms-win-crt-runtime-l1-1-0.dll
 0001:0000c050       __acrt_initialize          000000018000d050 f   MSVCRT:ucrt_stubs.obj
 0001:0000c050       __acrt_thread_attach       000000018000d050 f   MSVCRT:ucrt_stubs.obj
 0001:0000c050       __acrt_thread_detach       000000018000d050 f   MSVCRT:ucrt_stubs.obj
 0001:0000c050       __acrt_uninitialize        000000018000d050 f   MSVCRT:ucrt_stubs.obj
 0001:0000c050       __acrt_uninitialize_critical 000000018000d050 f   MSVCRT:ucrt_stubs.obj
 0001:0000c050       __scrt_stub_for_acrt_initialize 000000018000d050 f   MSVCRT:ucrt_stubs.obj
 0001:0000c050       __scrt_stub_for_acrt_thread_attach 000000018000d050 f   MSVCRT:ucrt_stubs.obj
 0001:0000c050       __scrt_stub_for_acrt_thread_detach 000000018000d050 f   MSVCRT:ucrt_stubs.obj
 0001:0000c050       __scrt_stub_for_acrt_uninitialize 000000018000d050 f   MSVCRT:ucrt_stubs.obj
 0001:0000c050       __scrt_stub_for_acrt_uninitialize_critical 000000018000d050 f   MSVCRT:ucrt_stubs.obj
 0001:0000c050       __vcrt_initialize          000000018000d050 f   MSVCRT:ucrt_stubs.obj
 0001:0000c050       __vcrt_thread_attach       000000018000d050 f   MSVCRT:ucrt_stubs.obj
 0001:0000c050       __vcrt_thread_detach       000000018000d050 f   MSVCRT:ucrt_stubs.obj
 0001:0000c050       __vcrt_uninitialize        000000018000d050 f   MSVCRT:ucrt_stubs.obj
 0001:0000c050       __vcrt_uninitialize_critical 000000018000d050 f   MSVCRT:ucrt_stubs.obj
 0001:0000c054       __scrt_stub_for_is_c_termination_complete 000000018000d054 f   MSVCRT:ucrt_stubs.obj
 0001:0000c054       _is_c_termination_complete 000000018000d054 f   MSVCRT:ucrt_stubs.obj
 0001:0000c070       _guard_dispatch_icall_nop  000000018000d070 f   MSVCRT:guard_dispatch.obj
 0001:0000c090       _guard_xfg_dispatch_icall_nop 000000018000d090 f   MSVCRT:guard_xfg_dispatch.obj
 0002:00000000       __imp_GetLastError         000000018000e000     kernel32:KERNEL32.dll
 0002:00000008       __imp_GetModuleHandleA     000000018000e008     kernel32:KERNEL32.dll
 0002:00000010       __imp_GetProcAddress       000000018000e010     kernel32:KERNEL32.dll
 0002:00000018       __imp_LoadLibraryA         000000018000e018     kernel32:KERNEL32.dll
 0002:00000020       __imp_LocalFree            000000018000e020     kernel32:KERNEL32.dll
 0002:00000028       __imp_FormatMessageA       000000018000e028     kernel32:KERNEL32.dll
 0002:00000030       __imp_FreeLibrary          000000018000e030     kernel32:KERNEL32.dll
 0002:00000038       __imp_RtlCaptureContext    000000018000e038     kernel32:KERNEL32.dll
 0002:00000040       __imp_RtlLookupFunctionEntry 000000018000e040     kernel32:KERNEL32.dll
 0002:00000048       __imp_RtlVirtualUnwind     000000018000e048     kernel32:KERNEL32.dll
 0002:00000050       __imp_UnhandledExceptionFilter 000000018000e050     kernel32:KERNEL32.dll
 0002:00000058       __imp_SetUnhandledExceptionFilter 000000018000e058     kernel32:KERNEL32.dll
 0002:00000060       __imp_GetCurrentProcess    000000018000e060     kernel32:KERNEL32.dll
 0002:00000068       __imp_TerminateProcess     000000018000e068     kernel32:KERNEL32.dll
 0002:00000070       __imp_IsProcessorFeaturePresent 000000018000e070     kernel32:KERNEL32.dll
 0002:00000078       __imp_QueryPerformanceCounter 000000018000e078     kernel32:KERNEL32.dll
 0002:00000080       __imp_GetCurrentProcessId  000000018000e080     kernel32:KERNEL32.dll
 0002:00000088       __imp_GetCurrentThreadId   000000018000e088     kernel32:KERNEL32.dll
 0002:00000090       __imp_GetSystemTimeAsFileTime 000000018000e090     kernel32:KERNEL32.dll
 0002:00000098       __imp_DisableThreadLibraryCalls 000000018000e098     kernel32:KERNEL32.dll
 0002:000000a0       __imp_InitializeSListHead  000000018000e0a0     kernel32:KERNEL32.dll
 0002:000000a8       __imp_IsDebuggerPresent    000000018000e0a8     kernel32:KERNEL32.dll
 0002:000000b0       \177KERNEL32_NULL_THUNK_DATA 000000018000e0b0     kernel32:KERNEL32.dll
 0002:000000b8       __imp_memcpy               000000018000e0b8     vcruntime:VCRUNTIME140.dll
 0002:000000c0       __imp_memset               000000018000e0c0     vcruntime:VCRUNTIME140.dll
 0002:000000c8       __imp___C_specific_handler 000000018000e0c8     vcruntime:VCRUNTIME140.dll
 0002:000000d0       __imp___std_type_info_destroy_list 000000018000e0d0     vcruntime:VCRUNTIME140.dll
 0002:000000d8       \177VCRUNTIME140_NULL_THUNK_DATA 000000018000e0d8     vcruntime:VCRUNTIME140.dll
 0002:000000e0       __imp_malloc               000000018000e0e0     ucrt:api-ms-win-crt-heap-l1-1-0.dll
 0002:000000e8       __imp_free                 000000018000e0e8     ucrt:api-ms-win-crt-heap-l1-1-0.dll
 0002:000000f0       __imp_calloc               000000018000e0f0     ucrt:api-ms-win-crt-heap-l1-1-0.dll
 0002:000000f8       \177api-ms-win-crt-heap-l1-1-0_NULL_THUNK_DATA 000000018000e0f8     ucrt:api-ms-win-crt-heap-l1-1-0.dll
 0002:00000100       __imp__cexit               000000018000e100     ucrt:api-ms-win-crt-runtime-l1-1-0.dll
 0002:00000108       __imp__execute_onexit_table 000000018000e108     ucrt:api-ms-win-crt-runtime-l1-1-0.dll
 0002:00000110       __imp__initialize_onexit_table 000000018000e110     ucrt:api-ms-win-crt-runtime-l1-1-0.dll
 0002:00000118       __imp__initialize_narrow_environment 000000018000e118     ucrt:api-ms-win-crt-runtime-l1-1-0.dll
 0002:00000120       __imp__initterm            000000018000e120     ucrt:api-ms-win-crt-runtime-l1-1-0.dll
 0002:00000128       __imp__initterm_e          000000018000e128     ucrt:api-ms-win-crt-runtime-l1-1-0.dll
 0002:00000130       __imp__seh_filter_dll      000000018000e130     ucrt:api-ms-win-crt-runtime-l1-1-0.dll
 0002:00000138       __imp__configure_narrow_argv 000000018000e138     ucrt:api-ms-win-crt-runtime-l1-1-0.dll
 0002:00000140       \177api-ms-win-crt-runtime-l1-1-0_NULL_THUNK_DATA 000000018000e140     ucrt:api-ms-win-crt-runtime-l1-1-0.dll
 0002:00000148       __imp_fflush               000000018000e148     ucrt:api-ms-win-crt-stdio-l1-1-0.dll
 0002:00000150       __imp___acrt_iob_func      000000018000e150     ucrt:api-ms-win-crt-stdio-l1-1-0.dll
 0002:00000158       __imp___stdio_common_vsprintf 000000018000e158     ucrt:api-ms-win-crt-stdio-l1-1-0.dll
 0002:00000160       __imp___stdio_common_vfprintf 000000018000e160     ucrt:api-ms-win-crt-stdio-l1-1-0.dll
 0002:00000168       \177api-ms-win-crt-stdio-l1-1-0_NULL_THUNK_DATA 000000018000e168     ucrt:api-ms-win-crt-stdio-l1-1-0.dll
 0002:00000170       __imp_strncmp              000000018000e170     ucrt:api-ms-win-crt-string-l1-1-0.dll
 0002:00000178       __imp_strlen               000000018000e178     ucrt:api-ms-win-crt-string-l1-1-0.dll
 0002:00000180       __imp_strcat               000000018000e180     ucrt:api-ms-win-crt-string-l1-1-0.dll
 0002:00000188       __imp_strcmp               000000018000e188     ucrt:api-ms-win-crt-string-l1-1-0.dll
 0002:00000190       __imp_strcpy               000000018000e190     ucrt:api-ms-win-crt-string-l1-1-0.dll
 0002:00000198       \177api-ms-win-crt-string-l1-1-0_NULL_THUNK_DATA 000000018000e198     ucrt:api-ms-win-crt-string-l1-1-0.dll
 0002:000001a0       __guard_check_icall_fptr   000000018000e1a0     MSVCRT:guard_support.obj
 0002:000001a8       __guard_xfg_check_icall_fptr 000000018000e1a8     MSVCRT:guard_support.obj
 0002:000001b0       __guard_dispatch_icall_fptr 000000018000e1b0     MSVCRT:guard_support.obj
 0002:000001b8       __guard_xfg_dispatch_icall_fptr 000000018000e1b8     MSVCRT:guard_support.obj
 0002:000001c0       __guard_xfg_table_dispatch_icall_fptr 000000018000e1c0     MSVCRT:guard_support.obj
 0002:000001c8       __castguard_check_failure_os_handled_fptr 000000018000e1c8     MSVCRT:guard_support.obj
 0002:000001d0       __guard_memcpy_fptr        000000018000e1d0     vcruntime:softmemtag.obj
 0002:000001d8       __xc_a                     000000018000e1d8     MSVCRT:initializers.obj
 0002:000001e0       __xc_z                     000000018000e1e0     MSVCRT:initializers.obj
 0002:000001e8       __xi_a                     000000018000e1e8     MSVCRT:initializers.obj
 0002:000001f0       __xi_z                     000000018000e1f0     MSVCRT:initializers.obj
 0002:000001f8       __xp_a                     000000018000e1f8     MSVCRT:initializers.obj
 0002:00000200       __xp_z                     000000018000e200     MSVCRT:initializers.obj
 0002:00000208       __xt_a                     000000018000e208     MSVCRT:initializers.obj
 0002:00000210       __xt_z                     000000018000e210     MSVCRT:initializers.obj
 0002:00000220       ??_C@_0BB@EFFKAOLB@NSS_VersionCheck@ 000000018000e220     j2secmod.obj
 0002:00000238       ??_C@_0P@JCBGNBMA@NSS_Initialize@ 000000018000e238     j2secmod.obj
 0002:00000248       ??_C@_09GOBCDJFC@secmod?4db@ 000000018000e248     j2secmod.obj
 0002:00000254       ??_C@_04DAEILJDJ@sql?3@    000000018000e254     j2secmod.obj
 0002:00000260       ??_C@_0L@EOEDJBCP@pkcs11?4txt@ 000000018000e260     j2secmod.obj
 0002:00000270       ??_C@_08LJKFHILM@NSS_Init@ 000000018000e270     j2secmod.obj
 0002:00000279       ??_C@_00CNPNBAHC@@         000000018000e279     j2secmod.obj
 0002:00000280       ??_C@_0BC@KONLDBJC@NSS_InitReadWrite@ 000000018000e280     j2secmod.obj
 0002:00000298       ??_C@_0O@LCPIEDLO@NSS_NoDB_Init@ 000000018000e298     j2secmod.obj
 0002:000002a8       ??_C@_0BM@FOILBMDH@SECMOD_GetDefaultModuleList@ 000000018000e2a8     j2secmod.obj
 0002:000002c8       ??_C@_0BE@GPOIDJOH@java?1util?1ArrayList@ 000000018000e2c8     j2secmod.obj
 0002:000002dc       ??_C@_03GAEACAIP@?$CI?$CJV@ 000000018000e2dc     j2secmod.obj
 0002:000002e0       ??_C@_06FALKBLGB@?$DMinit?$DO@ 000000018000e2e0     j2secmod.obj
 0002:000002e8       ??_C@_0BG@DHOOFEJE@?$CILjava?1lang?1Object?$DL?$CJZ@ 000000018000e2e8     j2secmod.obj
 0002:00000300       ??_C@_03BDGOHNNK@add@      000000018000e300     j2secmod.obj
 0002:00000308       ??_C@_0CC@KDFBHMNN@sun?1security?1pkcs11?1Secmod$Modu@ 000000018000e308     j2secmod.obj
 0002:00000330       ??_C@_0DM@JNKODIFA@?$CILjava?1lang?1String?$DLLjava?1lang?1S@ 000000018000e330     j2secmod.obj
 0002:00000370       ??_C@_0BF@BNLKGCGH@Symbol?5not?5found?3?5?$CFs@ 000000018000e370     j2secmod_md.obj
 0002:00000388       ??_C@_0CE@BDNBALGO@sun?1security?1pkcs11?1wrapper?1CK_@ 000000018000e388     p11_convert.obj
 0002:000003b0       ??_C@_09KCOLIFDD@?$CI?$FLC?$FLC?$FLC?$CJV@ 000000018000e3b0     p11_convert.obj
 0002:000003c0       ??_C@_0CH@FAGBPBAL@sun?1security?1pkcs11?1wrapper?1CK_@ 000000018000e3c0     p11_convert.obj
 0002:000003e8       ??_C@_05MNEAHDDF@?$CIII?$CJV@ 000000018000e3e8     p11_convert.obj
 0002:000003f0       ??_C@_0CM@LGADNNOP@sun?1security?1pkcs11?1wrapper?1CK_@ 000000018000e3f0     p11_convert.obj
 0002:00000420       ??_C@_07MDGBCFEE@?$CIJJJJ?$CJV@ 000000018000e420     p11_convert.obj
 0002:00000428       ??_C@_0CJ@KOKMKMLD@sun?1security?1pkcs11?1wrapper?1CK_@ 000000018000e428     p11_convert.obj
 0002:00000458       ??_C@_0BH@CPAPLJAG@?$CIJLjava?1lang?1Object?$DL?$CJV@ 000000018000e458     p11_convert.obj
 0002:00000470       ??_C@_01HMGJMAIH@B@        000000018000e470     p11_convert.obj
 0002:00000474       ??_C@_05FEBMJMCL@major@    000000018000e474     p11_convert.obj
 0002:0000047c       ??_C@_05OLAOEALN@minor@    000000018000e47c     p11_convert.obj
 0002:00000484       ??_C@_02LLADPLHK@?$FLC@    000000018000e484     p11_convert.obj
 0002:00000488       ??_C@_04JFPLDHAO@year@     000000018000e488     p11_convert.obj
 0002:00000490       ??_C@_05MEBAADFH@month@    000000018000e490     p11_convert.obj
 0002:00000498       ??_C@_03NNBHCDBP@day@      000000018000e498     p11_convert.obj
 0002:0000049c       ??_C@_01LELAEKIP@J@        000000018000e49c     p11_convert.obj
 0002:000004a0       ??_C@_04GPMDFGEJ@type@     000000018000e4a0     p11_convert.obj
 0002:000004a8       ??_C@_0BD@HMGGFBMH@Ljava?1lang?1Object?$DL@ 000000018000e4a8     p11_convert.obj
 0002:000004bc       ??_C@_06MLDODIFP@pValue@   000000018000e4bc     p11_convert.obj
 0002:000004c8       ??_C@_0DC@HGPFDFFP@Lsun?1security?1pkcs11?1wrapper?1CK@ 000000018000e4c8     p11_convert.obj
 0002:00000500       ??_C@_0L@KDDOOLLF@RandomInfo@ 000000018000e500     p11_convert.obj
 0002:00000510       ??_C@_0DA@MGBKDFKC@sun?1security?1pkcs11?1wrapper?1CK_@ 000000018000e510     p11_convert.obj
 0002:00000540       ??_C@_02KCBIMKDL@?$FLB@    000000018000e540     p11_convert.obj
 0002:00000548       ??_C@_0O@DPKEFPKK@pClientRandom@ 000000018000e548     p11_convert.obj
 0002:00000558       ??_C@_0O@BDHOCNNP@pServerRandom@ 000000018000e558     p11_convert.obj
 0002:00000568       ??_C@_0CJ@KHCANOHB@Lsun?1security?1pkcs11?1wrapper?1CK@ 000000018000e568     p11_convert.obj
 0002:00000598       ??_C@_08KFNBPFOP@pVersion@ 000000018000e598     p11_convert.obj
 0002:000005a8       ??_C@_0DN@HBKDAKMN@sun?1security?1pkcs11?1wrapper?1CK_@ 000000018000e5a8     p11_convert.obj
 0002:000005e8       ??_C@_0DO@JGMPNKLG@sun?1security?1pkcs11?1wrapper?1CK_@ 000000018000e5e8     p11_convert.obj
 0002:00000628       ??_C@_0BB@MMANIKKH@prfHashMechanism@ 000000018000e628     p11_convert.obj
 0002:00000640       ??_C@_0EJ@KDLPJNNJ@sun?1security?1pkcs11?1wrapper?1CK_@ 000000018000e640     p11_convert.obj
 0002:00000690       ??_C@_0N@GEGHOLAK@pSessionHash@ 000000018000e690     p11_convert.obj
 0002:000006a0       ??_C@_0CO@DCJBCFCB@sun?1security?1pkcs11?1wrapper?1CK_@ 000000018000e6a0     p11_convert.obj
 0002:000006d0       ??_C@_05HJNJEGNP@pSeed@    000000018000e6d0     p11_convert.obj
 0002:000006d8       ??_C@_06EEEIHGKI@pLabel@   000000018000e6d8     p11_convert.obj
 0002:000006e0       ??_C@_07KBCFNIDO@pOutput@  000000018000e6e0     p11_convert.obj
 0002:000006e8       ??_C@_0CO@NBPNNDEJ@sun?1security?1pkcs11?1wrapper?1CK_@ 000000018000e6e8     p11_convert.obj
 0002:00000718       ??_C@_0N@IEICAFHB@prfMechanism@ 000000018000e718     p11_convert.obj
 0002:00000728       ??_C@_0M@LJIINDHF@ulMacLength@ 000000018000e728     p11_convert.obj
 0002:00000738       ??_C@_0BB@BJFICNNC@ulServerOrClient@ 000000018000e738     p11_convert.obj
 0002:00000750       ??_C@_0CL@FNIJKDCI@sun?1security?1pkcs11?1wrapper?1CK_@ 000000018000e750     p11_convert.obj
 0002:0000077c       ??_C@_01POHCFINO@Z@        000000018000e77c     p11_convert.obj
 0002:00000780       ??_C@_08EEGALFCD@bExtract@ 000000018000e780     p11_convert.obj
 0002:00000790       ??_C@_07MAMBGKAC@bExpand@  000000018000e790     p11_convert.obj
 0002:00000798       ??_C@_0L@MMDCJBCD@ulSaltType@ 000000018000e798     p11_convert.obj
 0002:000007a4       ??_C@_05LDKIPIFG@pSalt@    000000018000e7a4     p11_convert.obj
 0002:000007b0       ??_C@_08IHLFOGPP@hSaltKey@ 000000018000e7b0     p11_convert.obj
 0002:000007bc       ??_C@_05GFDKCJGP@pInfo@    000000018000e7bc     p11_convert.obj
 0002:000007c8       ??_C@_0DK@PEIBCIFG@sun?1security?1pkcs11?1wrapper?1CK_@ 000000018000e7c8     p11_convert.obj
 0002:00000804       ??_C@_05EEOIKHBI@pData@    000000018000e804     p11_convert.obj
 0002:00000810       ??_C@_0BA@CKOIHILJ@ulMacSizeInBits@ 000000018000e810     p11_convert.obj
 0002:00000820       ??_C@_0BA@PELMFMAE@ulKeySizeInBits@ 000000018000e820     p11_convert.obj
 0002:00000830       ??_C@_0P@LDDDJGAG@ulIVSizeInBits@ 000000018000e830     p11_convert.obj
 0002:00000840       ??_C@_09OOHKLCMP@bIsExport@ 000000018000e840     p11_convert.obj
 0002:00000850       ??_C@_0DA@CCEPBHDJ@sun?1security?1pkcs11?1wrapper?1CK_@ 000000018000e850     p11_convert.obj
 0002:00000880       ??_C@_0DC@BBMMCKLB@Lsun?1security?1pkcs11?1wrapper?1CK@ 000000018000e880     p11_convert.obj
 0002:000008b8       ??_C@_0BF@ODGIPGLB@pReturnedKeyMaterial@ 000000018000e8b8     p11_convert.obj
 0002:000008d0       ??_C@_09JAFBLFBM@pIVClient@ 000000018000e8d0     p11_convert.obj
 0002:000008e0       ??_C@_09NPBDGOJP@pIVServer@ 000000018000e8e0     p11_convert.obj
 0002:000008f0       ??_C@_0DD@IELHHAPM@sun?1security?1pkcs11?1wrapper?1CK_@ 000000018000e8f0     p11_convert.obj
 0002:00000928       ??_C@_0DE@JIDMGMIB@sun?1security?1pkcs11?1wrapper?1CK_@ 000000018000e928     p11_convert.obj
 0002:00000960       ??_C@_0CO@CAAEDKFF@sun?1security?1pkcs11?1wrapper?1CK_@ 000000018000e960     p11_convert.obj
 0002:00000990       ??_C@_0O@FAFICCFK@ulCounterBits@ 000000018000e990     p11_convert.obj
 0002:000009a0       ??_C@_02BNOEFKLB@cb@       000000018000e9a0     p11_convert.obj
 0002:000009a8       ??_C@_0CK@NKNHHAJC@sun?1security?1pkcs11?1wrapper?1CK_@ 000000018000e9a8     p11_convert.obj
 0002:000009d4       ??_C@_02DONNAIDC@iv@       000000018000e9d4     p11_convert.obj
 0002:000009d8       ??_C@_03BFKFLPDB@aad@      000000018000e9d8     p11_convert.obj
 0002:000009e0       ??_C@_07LJAAJOFG@tagBits@  000000018000e9e0     p11_convert.obj
 0002:000009e8       ??_C@_0CK@GKAOADBA@sun?1security?1pkcs11?1wrapper?1CK_@ 000000018000e9e8     p11_convert.obj
 0002:00000a18       ??_C@_07LDPMHAML@dataLen@  000000018000ea18     p11_convert.obj
 0002:00000a20       ??_C@_05OOEDLKEB@nonce@    000000018000ea20     p11_convert.obj
 0002:00000a28       ??_C@_06PBGIHEKB@macLen@   000000018000ea28     p11_convert.obj
 0002:00000a30       ??_C@_0EA@NNBELOMA@sun?1security?1pkcs11?1wrapper?1CK_@ 000000018000ea30     p11_convert.obj
 0002:00000a70       ??_C@_0CI@ELKCPMM@No?5parameter?5support?5for?5this?5m@ 000000018000ea70     p11_convert.obj
 0002:00000a98       ??_C@_0DE@FNJOAKHM@sun?1security?1pkcs11?1wrapper?1CK_@ 000000018000ea98     p11_convert.obj
 0002:00000ad0       ??_C@_07NIDPGPFG@hashAlg@  000000018000ead0     p11_convert.obj
 0002:00000ad8       ??_C@_03GJMIBOLJ@mgf@      000000018000ead8     p11_convert.obj
 0002:00000adc       ??_C@_06OEKOLKIL@source@   000000018000eadc     p11_convert.obj
 0002:00000ae8       ??_C@_0M@NGABHANP@pSourceData@ 000000018000eae8     p11_convert.obj
 0002:00000af8       ??_C@_0CK@JAAGIPM@sun?1security?1pkcs11?1wrapper?1CK_@ 000000018000eaf8     p11_convert.obj
 0002:00000b28       ??_C@_0M@GGOAOMAD@pInitVector@ 000000018000eb28     p11_convert.obj
 0002:00000b38       ??_C@_09KKEKIPIM@pPassword@ 000000018000eb38     p11_convert.obj
 0002:00000b48       ??_C@_0M@HPDAPCKI@ulIteration@ 000000018000eb48     p11_convert.obj
 0002:00000b58       ??_C@_0CJ@EEABPKHL@sun?1security?1pkcs11?1wrapper?1CK_@ 000000018000eb58     p11_convert.obj
 0002:00000b88       ??_C@_09ONMFBHMB@mechanism@ 000000018000eb88     p11_convert.obj
 0002:00000b98       ??_C@_0L@JBCBPDO@pParameter@ 000000018000eb98     p11_convert.obj
 0002:00000ba8       ??_C@_0M@FGJAKHMC@pInitVektor@ 000000018000eba8     p11_convert.obj
 0002:00000bb8       ??_C@_0DC@OALCDCIB@sun?1security?1pkcs11?1wrapper?1CK_@ 000000018000ebb8     p11_convert.obj
 0002:00000bf0       ??_C@_0DD@HHCPFFPF@sun?1security?1pkcs11?1wrapper?1CK_@ 000000018000ebf0     p11_convert.obj
 0002:00000c28       ??_C@_0CK@JEIICANG@Unknown?5PBKD2?5mechanism?5paramet@ 000000018000ec28     p11_convert.obj
 0002:00000c58       ??_C@_0L@BGFAFLOD@saltSource@ 000000018000ec58     p11_convert.obj
 0002:00000c68       ??_C@_0BA@IHHAPGDC@pSaltSourceData@ 000000018000ec68     p11_convert.obj
 0002:00000c78       ??_C@_0L@LEIMKHLK@iterations@ 000000018000ec78     p11_convert.obj
 0002:00000c84       ??_C@_03NBFGPAGA@prf@      000000018000ec84     p11_convert.obj
 0002:00000c88       ??_C@_08BINOACIC@pPrfData@ 000000018000ec88     p11_convert.obj
 0002:00000c98       ??_C@_0DD@JKKJEEHE@sun?1security?1pkcs11?1wrapper?1CK_@ 000000018000ec98     p11_convert.obj
 0002:00000ccc       ??_C@_04ODAPDKJK@sLen@     000000018000eccc     p11_convert.obj
 0002:00000cd8       ??_C@_0DD@BKPMIPL@sun?1security?1pkcs11?1wrapper?1CK_@ 000000018000ecd8     p11_convert.obj
 0002:00000d0c       ??_C@_03EOOFPPDM@kdf@      000000018000ed0c     p11_convert.obj
 0002:00000d10       ??_C@_0M@GNHNJOEE@pSharedData@ 000000018000ed10     p11_convert.obj
 0002:00000d20       ??_C@_0M@KMNGLHAN@pPublicData@ 000000018000ed20     p11_convert.obj
 0002:00000d30       ??_C@_0DD@CIGHHMAJ@sun?1security?1pkcs11?1wrapper?1CK_@ 000000018000ed30     p11_convert.obj
 0002:00000d68       ??_C@_0BB@FHLLIPHA@ulPrivateDataLen@ 000000018000ed68     p11_convert.obj
 0002:00000d80       ??_C@_0N@MNKNKKOE@hPrivateData@ 000000018000ed80     p11_convert.obj
 0002:00000d90       ??_C@_0N@JDGNPOHL@pPublicData2@ 000000018000ed90     p11_convert.obj
 0002:00000da0       ??_C@_0DH@KLOKCPBP@sun?1security?1pkcs11?1wrapper?1CK_@ 000000018000eda0     p11_convert.obj
 0002:00000dd8       ??_C@_0L@BEOLNMGA@pOtherInfo@ 000000018000edd8     p11_convert.obj
 0002:00000de8       ??_C@_0DH@ICCCJLON@sun?1security?1pkcs11?1wrapper?1CK_@ 000000018000ede8     p11_convert.obj
 0002:00000e20       ??_C@_0M@KOOGEDPH@pNativeData@ 000000018000ee20     p11_general.obj
 0002:00000e30       ??_C@_0P@MLLHBNNC@java?1lang?1Long@ 000000018000ee30     p11_general.obj
 0002:00000e40       ??_C@_0CE@FGGPEABN@sun?1security?1pkcs11?1wrapper?1CK_@ 000000018000ee40     p11_general.obj
 0002:00000e70       ??_C@_0FJ@PCBLKCL@?$CILsun?1security?1pkcs11?1wrapper?1C@ 000000018000ee70     p11_general.obj
 0002:00000ed0       ??_C@_0CJ@BIOEJKNF@sun?1security?1pkcs11?1wrapper?1CK_@ 000000018000eed0     p11_general.obj
 0002:00000f00       ??_C@_0FJ@OBILFDMI@?$CI?$FLC?$FLCJLsun?1security?1pkcs11?1wrap@ 000000018000ef00     p11_general.obj
 0002:00000f60       ??_C@_0CK@MCNCOGLO@sun?1security?1pkcs11?1wrapper?1CK_@ 000000018000ef60     p11_general.obj
 0002:00000f90       ??_C@_0GJ@FDGHLOMM@?$CI?$FLC?$FLC?$FLC?$FLCJJJJJJJJJJJLsun?1securi@ 000000018000ef90     p11_general.obj
 0002:00001000       ??_C@_0CO@CCAIMKIH@sun?1security?1pkcs11?1wrapper?1CK_@ 000000018000f000     p11_general.obj
 0002:00001030       ??_C@_06NJFABHM@?$CIJJJ?$CJV@ 000000018000f030     p11_general.obj
 0002:00001040       ??_C@_0HA@JHHDDDM@C_1GenerateKeyPair?$CI?$CJ?3?5C_Generat@ 000000018000f040     p11_keymgmt.obj
 0002:000010b0       ??_C@_0BB@DDIADMEB@hClientMacSecret@ 000000018000f0b0     p11_keymgmt.obj
 0002:000010c8       ??_C@_0BB@BKLFLGGI@hServerMacSecret@ 000000018000f0c8     p11_keymgmt.obj
 0002:000010e0       ??_C@_0L@GFMHBDMC@hClientKey@ 000000018000f0e0     p11_keymgmt.obj
 0002:000010f0       ??_C@_0L@HMKKIKDM@hServerKey@ 000000018000f0f0     p11_keymgmt.obj
 0002:00001100       ??_C@_0P@DKECOBED@C_GetInterface@ 000000018000f100     p11_md.obj
 0002:00001110       ??_C@_0BC@GHFGDNNP@C_GetFunctionList@ 000000018000f110     p11_md.obj
 0002:00001128       ??_C@_0CC@IGCOJME@ERROR?3?5No?5function?5list?5ptr?5fou@ 000000018000f128     p11_md.obj
 0002:00001150       ??_C@_0DB@KELDKOFM@sun?1security?1pkcs11?1wrapper?1CK_@ 000000018000f150     p11_mutex.obj
 0002:00001188       ??_C@_0CN@MIBMAGA@Lsun?1security?1pkcs11?1wrapper?1CK@ 000000018000f188     p11_mutex.obj
 0002:000011b8       ??_C@_0M@CHIIKKKK@CreateMutex@ 000000018000f1b8     p11_mutex.obj
 0002:000011c8       ??_C@_0CO@KLPPKFHK@Lsun?1security?1pkcs11?1wrapper?1CK@ 000000018000f1c8     p11_mutex.obj
 0002:000011f8       ??_C@_0N@MEBBDPAH@DestroyMutex@ 000000018000f1f8     p11_mutex.obj
 0002:00001208       ??_C@_0CL@LBHOKNDM@Lsun?1security?1pkcs11?1wrapper?1CK@ 000000018000f208     p11_mutex.obj
 0002:00001238       ??_C@_09DKPDKGG@LockMutex@ 000000018000f238     p11_mutex.obj
 0002:00001248       ??_C@_0CN@KJNOCKKG@Lsun?1security?1pkcs11?1wrapper?1CK@ 000000018000f248     p11_mutex.obj
 0002:00001278       ??_C@_0M@HCNHAHIN@UnlockMutex@ 000000018000f278     p11_mutex.obj
 0002:00001284       ??_C@_05GECEPKB@flags@     000000018000f284     p11_mutex.obj
 0002:00001290       ??_C@_09CJOBGKOG@pReserved@ 000000018000f290     p11_mutex.obj
 0002:000012a0       ??_C@_0CL@FFENGHBF@sun?1security?1pkcs11?1wrapper?1CK_@ 000000018000f2a0     p11_mutex.obj
 0002:000012d0       ??_C@_0BF@LHBAMMHC@?$CI?$CJLjava?1lang?1Object?$DL@ 000000018000f2d0     p11_mutex.obj
 0002:000012e8       ??_C@_0P@MBLCOHGI@CK_CREATEMUTEX@ 000000018000f2e8     p11_mutex.obj
 0002:000012f8       ??_C@_0CM@EDGLGECO@sun?1security?1pkcs11?1wrapper?1PKC@ 000000018000f2f8     p11_mutex.obj
 0002:00001324       ??_C@_03IGDHHNNC@?$CI?$CJJ@ 000000018000f324     p11_mutex.obj
 0002:00001328       ??_C@_0N@CFOEEHFM@getErrorCode@ 000000018000f328     p11_mutex.obj
 0002:00001338       ??_C@_0CM@MCCIEMNP@sun?1security?1pkcs11?1wrapper?1CK_@ 000000018000f338     p11_mutex.obj
 0002:00001368       ??_C@_0BG@JLFLBLJI@?$CILjava?1lang?1Object?$DL?$CJV@ 000000018000f368     p11_mutex.obj
 0002:00001380       ??_C@_0BA@OMAILONO@CK_DESTROYMUTEX@ 000000018000f380     p11_mutex.obj
 0002:00001390       ??_C@_0CJ@OCJKNBDK@sun?1security?1pkcs11?1wrapper?1CK_@ 000000018000f390     p11_mutex.obj
 0002:000013c0       ??_C@_0N@DNKBOIPK@CK_LOCKMUTEX@ 000000018000f3c0     p11_mutex.obj
 0002:000013d0       ??_C@_0CL@BCMKDC@sun?1security?1pkcs11?1wrapper?1CK_@ 000000018000f3d0     p11_mutex.obj
 0002:00001400       ??_C@_0P@JEONEKEP@CK_UNLOCKMUTEX@ 000000018000f400     p11_mutex.obj
 0002:00001410       ??_C@_06MELFAPKK@?50x?$CFlX@ 000000018000f410     p11_objmgmt.obj
 0002:00001418       ??_C@_0CG@KHGOBKJJ@sun?1security?1pkcs11?1wrapper?1CK_@ 000000018000f418     p11_sessmgmt.obj
 0002:00001440       ??_C@_0BI@DIAMFDOH@?$CIJJLjava?1lang?1Object?$DL?$CJV@ 000000018000f440     p11_sessmgmt.obj
 0002:00001458       ??_C@_09GHOCIINE@CK_NOTIFY@ 000000018000f458     p11_sessmgmt.obj
 0002:00001468       ??_C@_0CK@GAEPNKCI@This?5object?5is?5not?5connected?5to@ 000000018000f468     p11_util.obj
 0002:00001498       ??_C@_0BB@DDFKOHA@java?1lang?1Object@ 000000018000f498     p11_util.obj
 0002:000014b0       ??_C@_0BH@DOGHFNPN@?$CIJLjava?1lang?1String?$DL?$CJV@ 000000018000f4b0     p11_util.obj
 0002:000014c8       ??_C@_0BL@ENCPOIKC@java?1lang?1OutOfMemoryError@ 000000018000f4c8     p11_util.obj
 0002:000014e8       ??_C@_0BP@GJLHLAKJ@java?1lang?1NullPointerException@ 000000018000f4e8     p11_util.obj
 0002:00001508       ??_C@_0BE@EBAPEBGJ@java?1io?1IOException@ 000000018000f508     p11_util.obj
 0002:00001520       ??_C@_0DD@DEDAKGI@sun?1security?1pkcs11?1wrapper?1PKC@ 000000018000f520     p11_util.obj
 0002:00001558       ??_C@_0BC@DDPBLLCP@java?1lang?1Boolean@ 000000018000f558     p11_util.obj
 0002:0000156c       ??_C@_04LHKBAEFM@?$CIZ?$CJV@ 000000018000f56c     p11_util.obj
 0002:00001574       ??_C@_04OHLIFDMD@?$CIJ?$CJV@ 000000018000f574     p11_util.obj
 0002:0000157c       ??_C@_03MMPFGPID@?$CI?$CJZ@ 000000018000f57c     p11_util.obj
 0002:00001580       ??_C@_0N@FIOMDIJC@booleanValue@ 000000018000f580     p11_util.obj
 0002:00001590       ??_C@_0P@CCHCOPNE@java?1lang?1Byte@ 000000018000f590     p11_util.obj
 0002:000015a0       ??_C@_03EOOOPHNK@?$CI?$CJB@ 000000018000f5a0     p11_util.obj
 0002:000015a8       ??_C@_09CBDGACJH@byteValue@ 000000018000f5a8     p11_util.obj
 0002:000015b8       ??_C@_0BC@OHJKABOO@java?1lang?1Integer@ 000000018000f5b8     p11_util.obj
 0002:000015cc       ??_C@_03KNBKCOBB@?$CI?$CJI@ 000000018000f5cc     p11_util.obj
 0002:000015d0       ??_C@_08HBLFFCOK@intValue@ 000000018000f5d0     p11_util.obj
 0002:000015e0       ??_C@_09JKMBDFBF@longValue@ 000000018000f5e0     p11_util.obj
 0002:000015f0       ??_C@_0P@OINJBDJD@java?1lang?1Char@ 000000018000f5f0     p11_util.obj
 0002:00001600       ??_C@_03FHPFMGJL@?$CI?$CJC@ 000000018000f600     p11_util.obj
 0002:00001608       ??_C@_09ODGNKCJE@charValue@ 000000018000f608     p11_util.obj
 0002:00001618       ??_C@_0BE@GKIHCGPM@java?1lang?1Character@ 000000018000f618     p11_util.obj
 0002:0000162c       ??_C@_02CAADFCGC@?$FLZ@    000000018000f62c     p11_util.obj
 0002:00001630       ??_C@_02EBOMBDPA@?$FLI@    000000018000f630     p11_util.obj
 0002:00001634       ??_C@_02GKMBEADD@?$FLJ@    000000018000f634     p11_util.obj
 0002:00001638       ??_C@_0BB@FLFAIHG@java?1lang?1String@ 000000018000f638     p11_util.obj
 0002:00001650       ??_C@_0BE@IIFEGCLG@?$CI?$CJLjava?1lang?1Class?$DL@ 000000018000f650     p11_util.obj
 0002:00001668       ??_C@_08KFOJNDAP@getClass@ 000000018000f668     p11_util.obj
 0002:00001678       ??_C@_0BA@JJLOPNCP@java?1lang?1Class@ 000000018000f678     p11_util.obj
 0002:00001688       ??_C@_0BF@FOHFOJOB@?$CI?$CJLjava?1lang?1String?$DL@ 000000018000f688     p11_util.obj
 0002:000016a0       ??_C@_07DFBCBEHO@getName@  000000018000f6a0     p11_util.obj
 0002:000016b0       ??_C@_0EH@CMCPFLGF@Java?5object?5of?5this?5class?5canno@ 000000018000f6b0     p11_util.obj
 0002:000016f8       ??_C@_0M@LFMBLMNP@sunpkcs11?3?5@ 000000018000f6f8     p11_util.obj
 0002:00001708       _pDefaultRawDllMain        000000018000f708     MSVCRT:dll_dllmain.obj
 0002:00001708       _pRawDllMain               000000018000f708     MSVCRT:dll_dllmain.obj
 0002:00001720       __xmm@ffffffffffffffffffffffffffffffff 000000018000f720     MSVCRT:utility.obj
 0002:00001730       _load_config_used          000000018000f730     MSVCRT:loadcfg.obj
 0002:00001900       __volatile_metadata        000000018000f900     <linker-defined>
 0002:00001c20       __rtc_iaa                  000000018000fc20     MSVCRT:initsect.obj
 0002:00001c28       __rtc_izz                  000000018000fc28     MSVCRT:initsect.obj
 0002:00001c30       __rtc_taa                  000000018000fc30     MSVCRT:initsect.obj
 0002:00001c38       __rtc_tzz                  000000018000fc38     MSVCRT:initsect.obj
 0002:00003548       __IMPORT_DESCRIPTOR_KERNEL32 0000000180011548     kernel32:KERNEL32.dll
 0002:0000355c       __IMPORT_DESCRIPTOR_VCRUNTIME140 000000018001155c     vcruntime:VCRUNTIME140.dll
 0002:00003570       __IMPORT_DESCRIPTOR_api-ms-win-crt-string-l1-1-0 0000000180011570     ucrt:api-ms-win-crt-string-l1-1-0.dll
 0002:00003584       __IMPORT_DESCRIPTOR_api-ms-win-crt-stdio-l1-1-0 0000000180011584     ucrt:api-ms-win-crt-stdio-l1-1-0.dll
 0002:00003598       __IMPORT_DESCRIPTOR_api-ms-win-crt-heap-l1-1-0 0000000180011598     ucrt:api-ms-win-crt-heap-l1-1-0.dll
 0002:000035ac       __IMPORT_DESCRIPTOR_api-ms-win-crt-runtime-l1-1-0 00000001800115ac     ucrt:api-ms-win-crt-runtime-l1-1-0.dll
 0002:000035c0       __NULL_IMPORT_DESCRIPTOR   00000001800115c0     kernel32:KERNEL32.dll
 0003:000003c0       __security_cookie          00000001800123c0     MSVCRT:gs_cookie.obj
 0003:000003c8       __security_cookie_complement 00000001800123c8     MSVCRT:gs_cookie.obj
 0003:000003d0       __scrt_native_dllmain_reason 00000001800123d0     MSVCRT:utility.obj
 0003:000003d8       __isa_available            00000001800123d8     MSVCRT:cpu_disp.obj
 0003:000003dc       __isa_enabled              00000001800123dc     MSVCRT:cpu_disp.obj
 0003:000003e0       __memset_fast_string_threshold 00000001800123e0     MSVCRT:cpu_disp.obj
 0003:000003e8       __memset_nt_threshold      00000001800123e8     MSVCRT:cpu_disp.obj
 0003:000003f0       __scrt_ucrt_dll_is_in_use  00000001800123f0     MSVCRT:ucrt_stubs.obj
 0003:00000400       jvm_j2pkcs11               0000000180012400     p11_general.obj
 0003:00000408       debug_j2pkcs11             0000000180012408     p11_general.obj
 0003:00000410       notifyListHead             0000000180012410     p11_sessmgmt.obj
 0003:00000418       notifyListLock             0000000180012418     p11_sessmgmt.obj
 0003:000009a0       ?__type_info_root_node@@3U__type_info_node@@A 00000001800129a0     MSVCRT:tncleanup.obj
 0003:000009b0       ?_OptionsStorage@?1??__local_stdio_scanf_options@@9@4_KA 00000001800129b0     MSVCRT:default_local_stdio_options.obj
 0003:000009b8       __scrt_current_native_startup_state 00000001800129b8     MSVCRT:utility.obj
 0003:000009c0       __scrt_native_startup_lock 00000001800129c0     MSVCRT:utility.obj
 0003:00000a00       __scrt_debugger_hook_flag  0000000180012a00     MSVCRT:utility_desktop.obj
 0003:00000a04       __favor                    0000000180012a04     MSVCRT:cpu_disp.obj
 0003:00000a08       ckpGlobalInitArgs          0000000180012a08     <common>
 0003:00000a10       jInitArgsObject            0000000180012a10     <common>
 0003:00000a18       jLongClass                 0000000180012a18     <common>
 0003:00000a20       jByteArrayClass            0000000180012a20     <common>
 0003:00000a28       mech_pParameterID          0000000180012a28     <common>
 0003:00000a30       mech_mechanismID           0000000180012a30     <common>
 0003:00000a38       pNativeDataID              0000000180012a38     <common>
 0003:00000a40       ?_OptionsStorage@?1??__local_stdio_printf_options@@9@9 0000000180012a40     <common>
 0003:00000a48       __dyn_tls_init_callback    0000000180012a48     <common>

 entry point at        0001:0000b660

 Static symbols

 0000:fffea000       .debug$S                   0000000180000000     j2pkcs11.exp
 0000:fffea000       .debug$S                   0000000180000000     vcruntime:VCRUNTIME140.dll
 0000:fffea000       .debug$S                   0000000180000000     vcruntime:VCRUNTIME140.dll
 0000:fffea000       .debug$S                   0000000180000000     vcruntime:VCRUNTIME140.dll
 0000:fffea000       .debug$S                   0000000180000000     vcruntime:VCRUNTIME140.dll
 0000:fffea000       .debug$S                   0000000180000000     vcruntime:VCRUNTIME140.dll
 0000:fffea000       .debug$S                   0000000180000000     vcruntime:VCRUNTIME140.dll
 0000:fffea000       .debug$S                   0000000180000000     ucrt:api-ms-win-crt-heap-l1-1-0.dll
 0000:fffea000       .debug$S                   0000000180000000     ucrt:api-ms-win-crt-heap-l1-1-0.dll
 0000:fffea000       .debug$S                   0000000180000000     ucrt:api-ms-win-crt-heap-l1-1-0.dll
 0000:fffea000       .debug$S                   0000000180000000     ucrt:api-ms-win-crt-runtime-l1-1-0.dll
 0000:fffea000       .debug$S                   0000000180000000     ucrt:api-ms-win-crt-runtime-l1-1-0.dll
 0000:fffea000       .debug$S                   0000000180000000     ucrt:api-ms-win-crt-runtime-l1-1-0.dll
 0000:fffea000       .debug$S                   0000000180000000     ucrt:api-ms-win-crt-runtime-l1-1-0.dll
 0000:fffea000       .debug$S                   0000000180000000     ucrt:api-ms-win-crt-runtime-l1-1-0.dll
 0000:fffea000       .debug$S                   0000000180000000     ucrt:api-ms-win-crt-runtime-l1-1-0.dll
 0000:fffea000       .debug$S                   0000000180000000     ucrt:api-ms-win-crt-runtime-l1-1-0.dll
 0000:fffea000       .debug$S                   0000000180000000     ucrt:api-ms-win-crt-runtime-l1-1-0.dll
 0000:fffea000       .debug$S                   0000000180000000     ucrt:api-ms-win-crt-runtime-l1-1-0.dll
 0000:fffea000       .debug$S                   0000000180000000     ucrt:api-ms-win-crt-runtime-l1-1-0.dll
 0000:fffea000       .debug$S                   0000000180000000     ucrt:api-ms-win-crt-runtime-l1-1-0.dll
 0000:fffea000       .debug$S                   0000000180000000     ucrt:api-ms-win-crt-runtime-l1-1-0.dll
 0000:fffea000       .debug$S                   0000000180000000     ucrt:api-ms-win-crt-stdio-l1-1-0.dll
 0000:fffea000       .debug$S                   0000000180000000     ucrt:api-ms-win-crt-stdio-l1-1-0.dll
 0000:fffea000       .debug$S                   0000000180000000     ucrt:api-ms-win-crt-stdio-l1-1-0.dll
 0000:fffea000       .debug$S                   0000000180000000     ucrt:api-ms-win-crt-stdio-l1-1-0.dll
 0000:fffea000       .debug$S                   0000000180000000     ucrt:api-ms-win-crt-string-l1-1-0.dll
 0000:fffea000       .debug$S                   0000000180000000     ucrt:api-ms-win-crt-string-l1-1-0.dll
 0000:fffea000       .debug$S                   0000000180000000     ucrt:api-ms-win-crt-string-l1-1-0.dll
 0000:fffea000       .debug$S                   0000000180000000     ucrt:api-ms-win-crt-string-l1-1-0.dll
 0000:fffea000       .debug$S                   0000000180000000     ucrt:api-ms-win-crt-string-l1-1-0.dll
 0000:fffea000       .debug$S                   0000000180000000     kernel32:KERNEL32.dll
 0000:fffea000       .debug$S                   0000000180000000     kernel32:KERNEL32.dll
 0000:fffea000       .debug$S                   0000000180000000     kernel32:KERNEL32.dll
 0000:fffea000       .debug$S                   0000000180000000     kernel32:KERNEL32.dll
 0000:fffea000       .debug$S                   0000000180000000     kernel32:KERNEL32.dll
 0000:fffea000       .debug$S                   0000000180000000     kernel32:KERNEL32.dll
 0000:fffea000       .debug$S                   0000000180000000     kernel32:KERNEL32.dll
 0000:fffea000       .debug$S                   0000000180000000     kernel32:KERNEL32.dll
 0000:fffea000       .debug$S                   0000000180000000     kernel32:KERNEL32.dll
 0000:fffea000       .debug$S                   0000000180000000     kernel32:KERNEL32.dll
 0000:fffea000       .debug$S                   0000000180000000     kernel32:KERNEL32.dll
 0000:fffea000       .debug$S                   0000000180000000     kernel32:KERNEL32.dll
 0000:fffea000       .debug$S                   0000000180000000     kernel32:KERNEL32.dll
 0000:fffea000       .debug$S                   0000000180000000     kernel32:KERNEL32.dll
 0000:fffea000       .debug$S                   0000000180000000     kernel32:KERNEL32.dll
 0000:fffea000       .debug$S                   0000000180000000     kernel32:KERNEL32.dll
 0000:fffea000       .debug$S                   0000000180000000     kernel32:KERNEL32.dll
 0000:fffea000       .debug$S                   0000000180000000     kernel32:KERNEL32.dll
 0000:fffea000       .debug$S                   0000000180000000     kernel32:KERNEL32.dll
 0000:fffea000       .debug$S                   0000000180000000     kernel32:KERNEL32.dll
 0000:fffea000       .debug$S                   0000000180000000     kernel32:KERNEL32.dll
 0000:fffea000       .debug$S                   0000000180000000     kernel32:KERNEL32.dll
 0000:fffea000       .debug$S                   0000000180000000     kernel32:KERNEL32.dll
 0000:fffea000       .debug$S                   0000000180000000     kernel32:KERNEL32.dll
 0001:00006bdc       copyBackClientVersion      0000000180007bdc f   p11_keymgmt.obj
 0001:00006da0       copyBackKeyMatParams       0000000180007da0 f   p11_keymgmt.obj
 0001:0000b0fc       throwByName                000000018000c0fc f   p11_util.obj
 0001:0000b2b0       $$000000                   000000018000c2b0     MSVCRT:amdsecgs.obj
 0001:0000b2e0       $$000000                   000000018000c2e0     MSVCRT:chkstk.obj
 0001:0000b340       ?dllmain_crt_dispatch@@YAHQEAUHINSTANCE__@@KQEAX@Z 000000018000c340 f   MSVCRT:dll_dllmain.obj
 0001:0000b390       ?dllmain_crt_process_attach@@YAHQEAUHINSTANCE__@@QEAX@Z 000000018000c390 f   MSVCRT:dll_dllmain.obj
 0001:0000b4a8       ?dllmain_crt_process_detach@@YAH_N@Z 000000018000c4a8 f   MSVCRT:dll_dllmain.obj
 0001:0000b52c       ?dllmain_dispatch@@YAHQEAUHINSTANCE__@@KQEAX@Z 000000018000c52c f   MSVCRT:dll_dllmain.obj
 0001:0000b7a8       capture_previous_context   000000018000c7a8 f   MSVCRT:gs_report.obj
 0001:0000c060       $$000000                   000000018000d060     MSVCRT:guard_dispatch.obj
 0001:0000c080       $$000000                   000000018000d080     MSVCRT:guard_xfg_dispatch.obj
 0001:0000c096       ?fin$0@?0??dllmain_crt_process_attach@@YAHQEAUHINSTANCE__@@QEAX@Z@4HA 000000018000d096 f   MSVCRT:dll_dllmain.obj
 0001:0000c0ad       ?fin$0@?0??dllmain_crt_process_detach@@YAH_N@Z@4HA 000000018000d0ad f   MSVCRT:dll_dllmain.obj
 0001:0000c0c6       ?fin$1@?0??dllmain_crt_process_detach@@YAH_N@Z@4HA 000000018000d0c6 f   MSVCRT:dll_dllmain.obj
 0001:0000c0da       ?filt$0@?0??dllmain_dispatch@@YAHQEAUHINSTANCE__@@KQEAX@Z@4HA 000000018000d0da f   MSVCRT:dll_dllmain.obj
 0001:0000c110       __scrt_is_nonwritable_in_current_image$filt$0 000000018000d110 f   MSVCRT:utility.obj
 0002:00001710       GS_ExceptionPointers       000000018000f710     MSVCRT:gs_report.obj
 0002:00001c40       $unwind$Java_sun_security_pkcs11_Secmod_nssVersionCheck 000000018000fc40     j2secmod.obj
 0002:00001c40       $unwind$Java_sun_security_pkcs11_Secmod_nssGetLibraryHandle 000000018000fc40     j2secmod_md.obj
 0002:00001c40       $unwind$jKeyDerivationStringDataToCKKeyDerivationStringDataPtr 000000018000fc40     p11_convert.obj
 0002:00001c40       $unwind$jMechParamToCKMechParamPtrSlow 000000018000fc40     p11_convert.obj
 0002:00001c40       $unwind$jMechanismToCKMechanismPtr 000000018000fc40     p11_convert.obj
 0002:00001c40       $unwind$jVersionToCKVersionPtr 000000018000fc40     p11_convert.obj
 0002:00001c40       $unwind$Java_sun_security_pkcs11_wrapper_PKCS11_C_1DecryptInit 000000018000fc40     p11_crypt.obj
 0002:00001c40       $unwind$Java_sun_security_pkcs11_wrapper_PKCS11_C_1EncryptInit 000000018000fc40     p11_crypt.obj
 0002:00001c40       $unwind$Java_sun_security_pkcs11_wrapper_PKCS11_C_1DigestInit 000000018000fc40     p11_digest.obj
 0002:00001c40       $unwind$Java_sun_security_pkcs11_wrapper_PKCS11_C_1Initialize 000000018000fc40     p11_general.obj
 0002:00001c40       $unwind$copyBackTLSPrfParams 000000018000fc40     p11_keymgmt.obj
 0002:00001c40       $unwind$Java_sun_security_pkcs11_wrapper_PKCS11_C_1SignInit 000000018000fc40     p11_sign.obj
 0002:00001c40       $unwind$Java_sun_security_pkcs11_wrapper_PKCS11_C_1SignRecoverInit 000000018000fc40     p11_sign.obj
 0002:00001c40       $unwind$Java_sun_security_pkcs11_wrapper_PKCS11_C_1VerifyInit 000000018000fc40     p11_sign.obj
 0002:00001c40       $unwind$Java_sun_security_pkcs11_wrapper_PKCS11_C_1VerifyRecoverInit 000000018000fc40     p11_sign.obj
 0002:00001c40       $unwind$ckBBoolPtrToJBooleanObject 000000018000fc40     p11_util.obj
 0002:00001c40       $unwind$__scrt_dllmain_exception_filter 000000018000fc40     MSVCRT:utility.obj
 0002:00001c54       $unwind$Java_sun_security_pkcs11_Secmod_nssInitialize 000000018000fc54     j2secmod.obj
 0002:00001c6c       $unwind$Java_sun_security_pkcs11_Secmod_nssGetModuleList 000000018000fc6c     j2secmod.obj
 0002:00001c88       $unwind$snprintf           000000018000fc88     j2secmod_md.obj
 0002:00001c98       $unwind$Java_sun_security_pkcs11_Secmod_nssLoadLibrary 000000018000fc98     j2secmod_md.obj
 0002:00001cac       $unwind$p11FindFunction    000000018000fcac     j2secmod_md.obj
 0002:00001cc4       $unwind$ckDatePtrToJDateObject 000000018000fcc4     p11_convert.obj
 0002:00001cc4       $unwind$jTls12MasterKeyDeriveParamToCKTls12MasterKeyDeriveParamPtr 000000018000fcc4     p11_convert.obj
 0002:00001cc4       $unwind$Java_sun_security_pkcs11_wrapper_PKCS11_C_1FindObjects 000000018000fcc4     p11_objmgmt.obj
 0002:00001cc4       $unwind$ckAssertReturnValueOK2 000000018000fcc4     p11_util.obj
 0002:00001cc4       $unwind$jAttributeArrayToCKAttributeArray 000000018000fcc4     p11_util.obj
 0002:00001cc4       $unwind$jBooleanArrayToCKBBoolArray 000000018000fcc4     p11_util.obj
 0002:00001cc4       $unwind$jCharArrayToCKCharArray 000000018000fcc4     p11_util.obj
 0002:00001cc4       $unwind$jCharArrayToCKUTF8CharArray 000000018000fcc4     p11_util.obj
 0002:00001cc4       $unwind$jLongArrayToCKULongArray 000000018000fcc4     p11_util.obj
 0002:00001cdc       $unwind$ckVersionPtrToJVersion 000000018000fcdc     p11_convert.obj
 0002:00001cdc       $unwind$ckMechanismInfoPtrToJMechanismInfo 000000018000fcdc     p11_general.obj
 0002:00001cec       $unwind$ckSessionInfoPtrToJSessionInfo 000000018000fcec     p11_convert.obj
 0002:00001cfc       $unwind$ckAttributePtrToJAttribute 000000018000fcfc     p11_convert.obj
 0002:00001cfc       $unwind$Java_sun_security_pkcs11_wrapper_PKCS11_C_1DecryptFinal 000000018000fcfc     p11_crypt.obj
 0002:00001cfc       $unwind$Java_sun_security_pkcs11_wrapper_PKCS11_C_1EncryptFinal 000000018000fcfc     p11_crypt.obj
 0002:00001cfc       $unwind$Java_sun_security_pkcs11_wrapper_PKCS11_C_1CreateObject 000000018000fcfc     p11_objmgmt.obj
 0002:00001cfc       $unwind$ckCharArrayToJCharArray 000000018000fcfc     p11_util.obj
 0002:00001cfc       $unwind$ckULongArrayToJLongArray 000000018000fcfc     p11_util.obj
 0002:00001cfc       $unwind$ckUTF8CharArrayToJCharArray 000000018000fcfc     p11_util.obj
 0002:00001cfc       $unwind$jByteArrayToCKByteArray 000000018000fcfc     p11_util.obj
 0002:00001d14       $unwind$jDateObjectToCKDatePtr 000000018000fd14     p11_convert.obj
 0002:00001d30       $unwind$jAttributeToCKAttribute 000000018000fd30     p11_convert.obj
 0002:00001d30       $unwind$jSalsaChaChaPolyParamsToCKSalsaChaChaPolyParamPtr 000000018000fd30     p11_convert.obj
 0002:00001d30       $unwind$copyBackClientVersion 000000018000fd30     p11_keymgmt.obj
 0002:00001d48       $unwind$jMechParamToCKMechParamPtr 000000018000fd48     p11_convert.obj
 0002:00001d48       $unwind$jObjectToPrimitiveCKObjectPtr 000000018000fd48     p11_util.obj
 0002:00001d5c       $unwind$jCCMParamsToCKCCMParamPtr 000000018000fd5c     p11_convert.obj
 0002:00001d5c       $unwind$jGCMParamsToCKGCMParamPtr 000000018000fd5c     p11_convert.obj
 0002:00001d5c       $unwind$jRsaPkcsOaepParamToCKRsaPkcsOaepParamPtr 000000018000fd5c     p11_convert.obj
 0002:00001d5c       $unwind$copyBackKeyMatParams 000000018000fd5c     p11_keymgmt.obj
 0002:00001d78       $unwind$jPbeParamToCKPbeParamPtr 000000018000fd78     p11_convert.obj
 0002:00001d90       $unwind$jEcdh2DeriveParamToCKEcdh2DeriveParamPtr 000000018000fd90     p11_convert.obj
 0002:00001d90       $unwind$jHkdfParamsToCKHkdfParamsPtr 000000018000fd90     p11_convert.obj
 0002:00001d90       $unwind$jPkcs5Pbkd2ParamToCKPkcs5Pbkd2ParamPtr 000000018000fd90     p11_convert.obj
 0002:00001da8       $unwind$jSsl3MasterKeyDeriveParamToCKSsl3MasterKeyDeriveParamPtr 000000018000fda8     p11_convert.obj
 0002:00001da8       $unwind$Java_sun_security_pkcs11_wrapper_PKCS11_C_1SeedRandom 000000018000fda8     p11_digest.obj
 0002:00001da8       $unwind$Java_sun_security_pkcs11_wrapper_PKCS11_C_1FindObjectsInit 000000018000fda8     p11_objmgmt.obj
 0002:00001da8       $unwind$Java_sun_security_pkcs11_wrapper_PKCS11_C_1SetAttributeValue 000000018000fda8     p11_objmgmt.obj
 0002:00001da8       $unwind$Java_sun_security_pkcs11_wrapper_PKCS11_C_1Login 000000018000fda8     p11_sessmgmt.obj
 0002:00001da8       $unwind$Java_sun_security_pkcs11_wrapper_PKCS11_C_1VerifyFinal 000000018000fda8     p11_sign.obj
 0002:00001da8       $unwind$ckByteArrayToJByteArray 000000018000fda8     p11_util.obj
 0002:00001dbc       $unwind$jSsl3KeyMatParamToCKSsl3KeyMatParamPtr 000000018000fdbc     p11_convert.obj
 0002:00001dd0       $unwind$copyBackPBEInitializationVector 000000018000fdd0     p11_convert.obj
 0002:00001dd0       $unwind$jEcdh1DeriveParamToCKEcdh1DeriveParamPtr 000000018000fdd0     p11_convert.obj
 0002:00001dd0       $unwind$jRsaPkcsPssParamToCKRsaPkcsPssParamPtr 000000018000fdd0     p11_convert.obj
 0002:00001dd0       $unwind$jTlsExtendedMasterKeyDeriveParamToCKTlsExtendedMasterKeyDeriveParamPtr 000000018000fdd0     p11_convert.obj
 0002:00001dd0       $unwind$jTlsMacParamsToCKTlsMacParamPtr 000000018000fdd0     p11_convert.obj
 0002:00001dd0       $unwind$jTlsPrfParamsToCKTlsPrfParamPtr 000000018000fdd0     p11_convert.obj
 0002:00001dd0       $unwind$jX942Dh1DeriveParamToCKX942Dh1DeriveParamPtr 000000018000fdd0     p11_convert.obj
 0002:00001dd0       $unwind$Java_sun_security_pkcs11_wrapper_PKCS11_C_1GCMDecryptInitWithRetry 000000018000fdd0     p11_crypt.obj
 0002:00001dd0       $unwind$Java_sun_security_pkcs11_wrapper_PKCS11_C_1GCMEncryptInitWithRetry 000000018000fdd0     p11_crypt.obj
 0002:00001dd0       $unwind$Java_sun_security_pkcs11_wrapper_PKCS11_C_1GenerateRandom 000000018000fdd0     p11_digest.obj
 0002:00001de8       $unwind$jX942Dh2DeriveParamToCKX942Dh2DeriveParamPtr 000000018000fde8     p11_convert.obj
 0002:00001e04       $unwind$masterKeyDeriveParamToCKMasterKeyDeriveParam 000000018000fe04     p11_convert.obj
 0002:00001e20       $unwind$keyMatParamToCKKeyMatParam 000000018000fe20     p11_convert.obj
 0002:00001e38       $unwind$jTls12KeyMatParamToCKTls12KeyMatParamPtr 000000018000fe38     p11_convert.obj
 0002:00001e50       $unwind$jAesCtrParamsToCKAesCtrParamPtr 000000018000fe50     p11_convert.obj
 0002:00001e64       $unwind$Java_sun_security_pkcs11_wrapper_PKCS11_C_1Decrypt 000000018000fe64     p11_crypt.obj
 0002:00001e64       $unwind$Java_sun_security_pkcs11_wrapper_PKCS11_C_1DecryptUpdate 000000018000fe64     p11_crypt.obj
 0002:00001e64       $unwind$Java_sun_security_pkcs11_wrapper_PKCS11_C_1Encrypt 000000018000fe64     p11_crypt.obj
 0002:00001e64       $unwind$Java_sun_security_pkcs11_wrapper_PKCS11_C_1EncryptUpdate 000000018000fe64     p11_crypt.obj
 0002:00001e7c       $unwind$Java_sun_security_pkcs11_wrapper_PKCS11_C_1DigestSingle 000000018000fe7c     p11_digest.obj
 0002:00001e9c       $unwind$Java_sun_security_pkcs11_wrapper_PKCS11_C_1DigestUpdate 000000018000fe9c     p11_digest.obj
 0002:00001e9c       $unwind$Java_sun_security_pkcs11_wrapper_PKCS11_C_1SignUpdate 000000018000fe9c     p11_sign.obj
 0002:00001e9c       $unwind$Java_sun_security_pkcs11_wrapper_PKCS11_C_1VerifyUpdate 000000018000fe9c     p11_sign.obj
 0002:00001ebc       $unwind$Java_sun_security_pkcs11_wrapper_PKCS11_C_1DigestKey 000000018000febc     p11_digest.obj
 0002:00001ebc       $unwind$Java_sun_security_pkcs11_wrapper_PKCS11_initializeLibrary 000000018000febc     p11_general.obj
 0002:00001ebc       $unwind$Java_sun_security_pkcs11_wrapper_PKCS11_C_1DestroyObject 000000018000febc     p11_objmgmt.obj
 0002:00001ebc       $unwind$Java_sun_security_pkcs11_wrapper_PKCS11_C_1SessionCancel 000000018000febc     p11_sessmgmt.obj
 0002:00001ebc       $unwind$removeNotifyEntry  000000018000febc     p11_sessmgmt.obj
 0002:00001ebc       $unwind$ckULongPtrToJLongObject 000000018000febc     p11_util.obj
 0002:00001ebc       $unwind$updateGCMParams    000000018000febc     p11_util.obj
 0002:00001ebc       $unwind$_DllMainCRTStartup 000000018000febc     MSVCRT:dll_dllmain.obj
 0002:00001ecc       $unwind$Java_sun_security_pkcs11_wrapper_PKCS11_C_1DigestFinal 000000018000fecc     p11_digest.obj
 0002:00001ee4       $unwind$Java_sun_security_pkcs11_wrapper_PKCS11_C_1Finalize 000000018000fee4     p11_general.obj
 0002:00001ee4       $unwind$prefetchFields     000000018000fee4     p11_general.obj
 0002:00001ee4       $unwind$Java_sun_security_pkcs11_wrapper_PKCS11_C_1FindObjectsFinal 000000018000fee4     p11_objmgmt.obj
 0002:00001ee4       $unwind$Java_sun_security_pkcs11_wrapper_PKCS11_C_1CloseSession 000000018000fee4     p11_sessmgmt.obj
 0002:00001ee4       $unwind$Java_sun_security_pkcs11_wrapper_PKCS11_C_1Logout 000000018000fee4     p11_sessmgmt.obj
 0002:00001ee4       $unwind$createLockObject   000000018000fee4     p11_util.obj
 0002:00001ee4       $unwind$jBooleanObjectToCKBBoolPtr 000000018000fee4     p11_util.obj
 0002:00001ee4       $unwind$jByteObjectToCKBytePtr 000000018000fee4     p11_util.obj
 0002:00001ee4       $unwind$jCharObjectToCKCharPtr 000000018000fee4     p11_util.obj
 0002:00001ee4       $unwind$jIntegerObjectToCKULongPtr 000000018000fee4     p11_util.obj
 0002:00001ee4       $unwind$jLongObjectToCKULongPtr 000000018000fee4     p11_util.obj
 0002:00001ee4       $unwind$throwByName        000000018000fee4     p11_util.obj
 0002:00001ee4       $unwind$_RTC_Initialize    000000018000fee4     MSVCRT:initsect.obj
 0002:00001ee4       $unwind$_RTC_Terminate     000000018000fee4     MSVCRT:initsect.obj
 0002:00001ef0       $unwind$Java_sun_security_pkcs11_wrapper_PKCS11_C_1GetInfo 000000018000fef0     p11_general.obj
 0002:00001f08       $unwind$Java_sun_security_pkcs11_wrapper_PKCS11_C_1GetMechanismList 000000018000ff08     p11_general.obj
 0002:00001f08       $unwind$Java_sun_security_pkcs11_wrapper_PKCS11_C_1GetSlotList 000000018000ff08     p11_general.obj
 0002:00001f08       $unwind$Java_sun_security_pkcs11_wrapper_PKCS11_C_1GetOperationState 000000018000ff08     p11_sessmgmt.obj
 0002:00001f1c       $unwind$Java_sun_security_pkcs11_wrapper_PKCS11_C_1GetSlotInfo 000000018000ff1c     p11_general.obj
 0002:00001f34       $unwind$Java_sun_security_pkcs11_wrapper_PKCS11_C_1GetTokenInfo 000000018000ff34     p11_general.obj
 0002:00001f4c       $unwind$Java_sun_security_pkcs11_wrapper_PKCS11_C_1GetMechanismInfo 000000018000ff4c     p11_general.obj
 0002:00001f64       $unwind$ckInfoPtrToJInfo   000000018000ff64     p11_general.obj
 0002:00001f64       $unwind$ckSlotInfoPtrToJSlotInfo 000000018000ff64     p11_general.obj
 0002:00001f80       $unwind$ckTokenInfoPtrToJTokenInfo 000000018000ff80     p11_general.obj
 0002:00001f9c       $unwind$fetchClass         000000018000ff9c     p11_general.obj
 0002:00001f9c       $unwind$getFunctionList    000000018000ff9c     p11_util.obj
 0002:00001f9c       $unwind$getFunctionList30  000000018000ff9c     p11_util.obj
 0002:00001f9c       $unwind$__raise_securityfailure 000000018000ff9c     MSVCRT:gs_report.obj
 0002:00001f9c       $unwind$__scrt_initialize_crt 000000018000ff9c     MSVCRT:utility.obj
 0002:00001f9c       $unwind$__scrt_initialize_onexit_tables 000000018000ff9c     MSVCRT:utility.obj
 0002:00001f9c       $unwind$__scrt_release_startup_lock 000000018000ff9c     MSVCRT:utility.obj
 0002:00001f9c       $unwind$__scrt_uninitialize_crt 000000018000ff9c     MSVCRT:utility.obj
 0002:00001fa4       $unwind$ssl3CopyBackKeyMatParams 000000018000ffa4     p11_keymgmt.obj
 0002:00001fa4       $unwind$tls12CopyBackKeyMatParams 000000018000ffa4     p11_keymgmt.obj
 0002:00001fac       $unwind$Java_sun_security_pkcs11_wrapper_PKCS11_getNativeKeyInfo 000000018000ffac     p11_keymgmt.obj
 0002:00001fcc       $unwind$Java_sun_security_pkcs11_wrapper_PKCS11_createNativeKey 000000018000ffcc     p11_keymgmt.obj
 0002:00001fe4       $unwind$Java_sun_security_pkcs11_wrapper_PKCS11_C_1GenerateKey 000000018000ffe4     p11_keymgmt.obj
 0002:00001ffc       $unwind$Java_sun_security_pkcs11_wrapper_PKCS11_C_1GenerateKeyPair 000000018000fffc     p11_keymgmt.obj
 0002:00002014       $unwind$Java_sun_security_pkcs11_wrapper_PKCS11_C_1WrapKey 0000000180010014     p11_keymgmt.obj
 0002:00002030       $unwind$Java_sun_security_pkcs11_wrapper_PKCS11_C_1UnwrapKey 0000000180010030     p11_keymgmt.obj
 0002:00002048       $unwind$Java_sun_security_pkcs11_wrapper_PKCS11_C_1DeriveKey 0000000180010048     p11_keymgmt.obj
 0002:00002064       $unwind$Java_sun_security_pkcs11_wrapper_PKCS11_connect 0000000180010064     p11_md.obj
 0002:0000207c       $unwind$Java_sun_security_pkcs11_wrapper_PKCS11_disconnect 000000018001007c     p11_md.obj
 0002:00002084       $unwind$makeCKInitArgsAdapter 0000000180010084     p11_mutex.obj
 0002:00002098       $unwind$callJCreateMutex   0000000180010098     p11_mutex.obj
 0002:00002098       $unwind$callJDestroyMutex  0000000180010098     p11_mutex.obj
 0002:00002098       $unwind$callJLockMutex     0000000180010098     p11_mutex.obj
 0002:00002098       $unwind$callJUnlockMutex   0000000180010098     p11_mutex.obj
 0002:000020b0       $unwind$Java_sun_security_pkcs11_wrapper_PKCS11_C_1CopyObject 00000001800100b0     p11_objmgmt.obj
 0002:000020c8       $unwind$Java_sun_security_pkcs11_wrapper_PKCS11_C_1GetAttributeValue 00000001800100c8     p11_objmgmt.obj
 0002:000020e4       $unwind$notifyCallback     00000001800100e4     p11_sessmgmt.obj
 0002:000020f8       $unwind$putNotifyEntry     00000001800100f8     p11_sessmgmt.obj
 0002:0000210c       $unwind$Java_sun_security_pkcs11_wrapper_PKCS11_C_1OpenSession 000000018001010c     p11_sessmgmt.obj
 0002:00002124       $unwind$Java_sun_security_pkcs11_wrapper_PKCS11_C_1GetSessionInfo 0000000180010124     p11_sessmgmt.obj
 0002:00002138       $unwind$Java_sun_security_pkcs11_wrapper_PKCS11_C_1SetOperationState 0000000180010138     p11_sessmgmt.obj
 0002:0000214c       $unwind$Java_sun_security_pkcs11_wrapper_PKCS11_C_1Sign 000000018001014c     p11_sign.obj
 0002:00002168       $unwind$Java_sun_security_pkcs11_wrapper_PKCS11_C_1SignFinal 0000000180010168     p11_sign.obj
 0002:00002184       $unwind$Java_sun_security_pkcs11_wrapper_PKCS11_C_1SignRecover 0000000180010184     p11_sign.obj
 0002:00002184       $unwind$Java_sun_security_pkcs11_wrapper_PKCS11_C_1VerifyRecover 0000000180010184     p11_sign.obj
 0002:000021a4       $unwind$Java_sun_security_pkcs11_wrapper_PKCS11_C_1Verify 00000001800101a4     p11_sign.obj
 0002:000021bc       $unwind$fprintf            00000001800101bc     p11_util.obj
 0002:000021c8       $unwind$printDebug         00000001800101c8     p11_util.obj
 0002:000021d4       $unwind$freeCKAttributeArray 00000001800101d4     p11_util.obj
 0002:000021e4       $unwind$freeCKMechanismPtr 00000001800101e4     p11_util.obj
 0002:000021f0       $unwind$jStringToCKUTF8CharArray 00000001800101f0     p11_util.obj
 0002:00002204       $unwind$putModuleEntry     0000000180010204     p11_util.obj
 0002:00002204       $unwind$__scrt_initialize_default_local_stdio_options 0000000180010204     MSVCRT:default_local_stdio_options.obj
 0002:00002204       $unwind$?dllmain_crt_dispatch@@YAHQEAUHINSTANCE__@@KQEAX@Z 0000000180010204     MSVCRT:dll_dllmain.obj
 0002:00002204       $unwind$DllMain            0000000180010204     MSVCRT:dll_dllmain_stub.obj
 0002:00002204       $unwind$__GSHandlerCheck   0000000180010204     MSVCRT:gshandler.obj
 0002:00002204       $unwind$__scrt_acquire_startup_lock 0000000180010204     MSVCRT:utility.obj
 0002:00002204       $unwind$__scrt_dllmain_after_initialize_c 0000000180010204     MSVCRT:utility.obj
 0002:00002204       $unwind$__scrt_dllmain_before_initialize_c 0000000180010204     MSVCRT:utility.obj
 0002:00002204       $unwind$__scrt_dllmain_crt_thread_attach 0000000180010204     MSVCRT:utility.obj
 0002:00002204       $unwind$__scrt_dllmain_crt_thread_detach 0000000180010204     MSVCRT:utility.obj
 0002:00002204       $unwind$__scrt_dllmain_uninitialize_c 0000000180010204     MSVCRT:utility.obj
 0002:00002204       $unwind$__scrt_dllmain_uninitialize_critical 0000000180010204     MSVCRT:utility.obj
 0002:0000220c       $unwind$__GSHandlerCheckCommon 000000018001020c     MSVCRT:gshandler.obj
 0002:00002218       $xdatasym                  0000000180010218     MSVCRT:amdsecgs.obj
 0002:00002220       $xdatasym                  0000000180010220     MSVCRT:chkstk.obj
 0002:00002228       $unwind$?dllmain_crt_process_attach@@YAHQEAUHINSTANCE__@@QEAX@Z 0000000180010228     MSVCRT:dll_dllmain.obj
 0002:00002264       $unwind$?fin$0@?0??dllmain_crt_process_attach@@YAHQEAUHINSTANCE__@@QEAX@Z@4HA 0000000180010264     MSVCRT:dll_dllmain.obj
 0002:00002264       $unwind$?fin$0@?0??dllmain_crt_process_detach@@YAH_N@Z@4HA 0000000180010264     MSVCRT:dll_dllmain.obj
 0002:00002264       $unwind$?fin$1@?0??dllmain_crt_process_detach@@YAH_N@Z@4HA 0000000180010264     MSVCRT:dll_dllmain.obj
 0002:0000226c       $unwind$?dllmain_crt_process_detach@@YAH_N@Z 000000018001026c     MSVCRT:dll_dllmain.obj
 0002:000022c0       $unwind$?dllmain_dispatch@@YAHQEAUHINSTANCE__@@KQEAX@Z 00000001800102c0     MSVCRT:dll_dllmain.obj
 0002:000022e8       $unwind$?filt$0@?0??dllmain_dispatch@@YAHQEAUHINSTANCE__@@KQEAX@Z@4HA 00000001800102e8     MSVCRT:dll_dllmain.obj
 0002:000022f0       $unwind$__report_gsfailure 00000001800102f0     MSVCRT:gs_report.obj
 0002:000022f8       $unwind$capture_previous_context 00000001800102f8     MSVCRT:gs_report.obj
 0002:00002304       $unwind$__security_init_cookie 0000000180010304     MSVCRT:gs_support.obj
 0002:00002310       $unwind$__scrt_is_nonwritable_in_current_image 0000000180010310     MSVCRT:utility.obj
 0002:00002330       $unwind$__scrt_is_nonwritable_in_current_image$filt$0 0000000180010330     MSVCRT:utility.obj
 0002:00002338       $unwind$__scrt_fastfail    0000000180010338     MSVCRT:utility_desktop.obj
 0002:00002348       $unwind$__isa_available_init 0000000180010348     MSVCRT:cpu_disp.obj
 0002:00002358       $xdatasym                  0000000180010358     MSVCRT:guard_dispatch.obj
 0002:00002360       $xdatasym                  0000000180010360     MSVCRT:guard_xfg_dispatch.obj
 0002:00002370       .edata                     0000000180010370     j2pkcs11.exp
 0002:00002398       rgpv                       0000000180010398     j2pkcs11.exp
 0002:000024b0       rgszName                   00000001800104b0     j2pkcs11.exp
 0002:000025c8       rgwOrd                     00000001800105c8     j2pkcs11.exp
 0002:00002654       szName                     0000000180010654     j2pkcs11.exp
 0002:00002661       $N00001                    0000000180010661     j2pkcs11.exp
 0002:0000266c       $N00002                    000000018001066c     j2pkcs11.exp
 0002:000026a0       $N00003                    00000001800106a0     j2pkcs11.exp
 0002:000026d1       $N00004                    00000001800106d1     j2pkcs11.exp
 0002:000026ff       $N00005                    00000001800106ff     j2pkcs11.exp
 0002:0000272e       $N00006                    000000018001072e     j2pkcs11.exp
 0002:0000275e       $N00007                    000000018001075e     j2pkcs11.exp
 0002:00002796       $N00008                    0000000180010796     j2pkcs11.exp
 0002:000027cc       $N00009                    00000001800107cc     j2pkcs11.exp
 0002:00002804       $N00010                    0000000180010804     j2pkcs11.exp
 0002:00002837       $N00011                    0000000180010837     j2pkcs11.exp
 0002:0000286f       $N00012                    000000018001086f     j2pkcs11.exp
 0002:000028a6       $N00013                    00000001800108a6     j2pkcs11.exp
 0002:000028df       $N00014                    00000001800108df     j2pkcs11.exp
 0002:00002914       $N00015                    0000000180010914     j2pkcs11.exp
 0002:0000294d       $N00016                    000000018001094d     j2pkcs11.exp
 0002:00002984       $N00017                    0000000180010984     j2pkcs11.exp
 0002:000029ba       $N00018                    00000001800109ba     j2pkcs11.exp
 0002:000029ef       $N00019                    00000001800109ef     j2pkcs11.exp
 0002:00002a27       $N00020                    0000000180010a27     j2pkcs11.exp
 0002:00002a5f       $N00021                    0000000180010a5f     j2pkcs11.exp
 0002:00002a92       $N00022                    0000000180010a92     j2pkcs11.exp
 0002:00002aca       $N00023                    0000000180010aca     j2pkcs11.exp
 0002:00002b01       $N00024                    0000000180010b01     j2pkcs11.exp
 0002:00002b3a       $N00025                    0000000180010b3a     j2pkcs11.exp
 0002:00002b6e       $N00026                    0000000180010b6e     j2pkcs11.exp
 0002:00002ba5       $N00027                    0000000180010ba5     j2pkcs11.exp
 0002:00002be1       $N00028                    0000000180010be1     j2pkcs11.exp
 0002:00002c1c       $N00029                    0000000180010c1c     j2pkcs11.exp
 0002:00002c5f       $N00030                    0000000180010c5f     j2pkcs11.exp
 0002:00002ca2       $N00031                    0000000180010ca2     j2pkcs11.exp
 0002:00002cd9       $N00032                    0000000180010cd9     j2pkcs11.exp
 0002:00002d14       $N00033                    0000000180010d14     j2pkcs11.exp
 0002:00002d4e       $N00034                    0000000180010d4e     j2pkcs11.exp
 0002:00002d8b       $N00035                    0000000180010d8b     j2pkcs11.exp
 0002:00002dbe       $N00036                    0000000180010dbe     j2pkcs11.exp
 0002:00002dfa       $N00037                    0000000180010dfa     j2pkcs11.exp
 0002:00002e36       $N00038                    0000000180010e36     j2pkcs11.exp
 0002:00002e73       $N00039                    0000000180010e73     j2pkcs11.exp
 0002:00002ead       $N00040                    0000000180010ead     j2pkcs11.exp
 0002:00002ee4       $N00041                    0000000180010ee4     j2pkcs11.exp
 0002:00002f1b       $N00042                    0000000180010f1b     j2pkcs11.exp
 0002:00002f53       $N00043                    0000000180010f53     j2pkcs11.exp
 0002:00002f89       $N00044                    0000000180010f89     j2pkcs11.exp
 0002:00002fba       $N00045                    0000000180010fba     j2pkcs11.exp
 0002:00002fec       $N00046                    0000000180010fec     j2pkcs11.exp
 0002:00003023       $N00047                    0000000180011023     j2pkcs11.exp
 0002:00003059       $N00048                    0000000180011059     j2pkcs11.exp
 0002:00003092       $N00049                    0000000180011092     j2pkcs11.exp
 0002:000030cf       $N00050                    00000001800110cf     j2pkcs11.exp
 0002:0000310c       $N00051                    000000018001110c     j2pkcs11.exp
 0002:0000313c       $N00052                    000000018001113c     j2pkcs11.exp
 0002:00003171       $N00053                    0000000180011171     j2pkcs11.exp
 0002:000031a5       $N00054                    00000001800111a5     j2pkcs11.exp
 0002:000031dc       $N00055                    00000001800111dc     j2pkcs11.exp
 0002:00003217       $N00056                    0000000180011217     j2pkcs11.exp
 0002:0000324d       $N00057                    000000018001124d     j2pkcs11.exp
 0002:00003282       $N00058                    0000000180011282     j2pkcs11.exp
 0002:000032b4       $N00059                    00000001800112b4     j2pkcs11.exp
 0002:000032eb       $N00060                    00000001800112eb     j2pkcs11.exp
 0002:00003321       $N00061                    0000000180011321     j2pkcs11.exp
 0002:0000335a       $N00062                    000000018001135a     j2pkcs11.exp
 0002:00003397       $N00063                    0000000180011397     j2pkcs11.exp
 0002:000033cf       $N00064                    00000001800113cf     j2pkcs11.exp
 0002:00003402       $N00065                    0000000180011402     j2pkcs11.exp
 0002:00003432       $N00066                    0000000180011432     j2pkcs11.exp
 0002:0000346a       $N00067                    000000018001146a     j2pkcs11.exp
 0002:0000349d       $N00068                    000000018001149d     j2pkcs11.exp
 0002:000034d5       $N00069                    00000001800114d5     j2pkcs11.exp
 0002:0000350e       $N00070                    000000018001150e     j2pkcs11.exp
 0002:00003950       .idata$6                   0000000180011950     kernel32:KERNEL32.dll
 0002:000039aa       .idata$6                   00000001800119aa     vcruntime:VCRUNTIME140.dll
 0002:00003b00       .idata$6                   0000000180011b00     ucrt:api-ms-win-crt-string-l1-1-0.dll
 0002:00003b22       .idata$6                   0000000180011b22     ucrt:api-ms-win-crt-stdio-l1-1-0.dll
 0002:00003b42       .idata$6                   0000000180011b42     ucrt:api-ms-win-crt-heap-l1-1-0.dll
 0002:00003b62       .idata$6                   0000000180011b62     ucrt:api-ms-win-crt-runtime-l1-1-0.dll
 0003:00000000       ckpAttributesTemplate      0000000180012000     p11_keymgmt.obj
 0003:00000420       ?__proc_attached@@3HA      0000000180012420     MSVCRT:dll_dllmain.obj
 0003:00000430       GS_ExceptionRecord         0000000180012430     MSVCRT:gs_report.obj
 0003:000004d0       GS_ContextRecord           00000001800124d0     MSVCRT:gs_report.obj
 0003:000009c8       ?is_initialized_as_dll@@3_NA 00000001800129c8     MSVCRT:utility.obj
 0003:000009c9       ?module_local_atexit_table_initialized@@3_NA 00000001800129c9     MSVCRT:utility.obj
 0003:000009d0       ?module_local_atexit_table@@3U_onexit_table_t@@A 00000001800129d0     MSVCRT:utility.obj
 0003:000009e8       ?module_local_at_quick_exit_table@@3U_onexit_table_t@@A 00000001800129e8     MSVCRT:utility.obj
 0005:00000060       $R000000                   0000000180014060     j2pkcs11.dll.res
